:06000000D3EF06F0120030
:0600080004EF08F01200F5
:100018000CEF08F012001DEE00F02DEE00F0F86A6B
:06002800EFEF06F01200EC
:1000300000001E0E126E136A7C0E146E156A166A8C
:1000400019681A681B68186A1200D9CFE6FFE1CF59
:10005000D9FFE65216501EE1040108BF1AD0400E27
:10006000E66E600EE66E000EE66E97EC06F0E55268
:10007000E552E552010E166EDF6A400EDF5C09E2C2
:10008000DF50EA6AA00FE96E000EEA22EF6ADF2A6B
:10009000F4D719D100016051080A01E10FD10F0A0C
:1000A00001E1D5D0010A01E1CCD0030A69E0010ADF
:1000B0005AE0070A45E0010A01E005D10001020EFD
:1000C000A06F00013A0EA16F0001010EA26F0001A6
:1000D000010EA36F0001A46B100EA56FA66BA76B9A
:1000E00013C0A8F014C0A9F015C0AAF0100E0001AA
:1000F000A95F000E0001AA5B0001AB6B0001030EBB
:10010000AC6F0001F80EAD6F7F0EAE6FAF6BB06BD2
:100110000001080EB16FB26BB36BB46B0001B5692F
:1001200004010CBF0CD0400EE66EA00EE66E000E71
:10013000E66E5DEC06F0E552E552E552166AC3D074
:100140000001615108E11F0E126EF80E136E7F0E52
:10015000146E156A06D01E0E126E136A7C0E146E93
:10016000156A166AB0D0040E176E1228175C06E2E4
:100170000400AED8F2EC04F0172AF7D7166AA3D021
:10018000E868191805E1E8681A1802E1E8681B1820
:1001900006E161C019F062C01AF063C01BF019508B
:1001A0000001611908E11A500001621904E11B50B5
:1001B0000001631900E143E1DF6A00016551DF5C82
:1001C0003EE2000E195C100E1A58000E1B582CE36C
:1001D00012285C6E5D6A0A0ED8905C365D36E806C1
:1001E000FBE15E6A5DBE5E685C50195C5D501A584A
:1001F0005E501B5819E23A0E0001D8806555DF2485
:10020000EA6A660FE96E000EEA22EF50E66E1850B9
:10021000E96EEA6AE9BEEA681C0EE926000EEA22E7
:10022000E552E750EF6E182A192A000E1A22000E26
:100230001B223A0E185C01E15ED8DF2ABED7166A8F
:1002400042D059D819681A681B68166A3CD0000158
:10025000070EA06F61C0A1F062C0A2F063C0A3F05E
:1002600064C0A4F065C0A5F061C0F6FF62C0F7FFEE
:1002700063C0F8FFDF6A00016551DF5C0FE209002F
:100280003A0E0001D8806555DF24EA6AA60FE96EB0
:10029000000EEA22F5CFEFFFDF2AEDD704010CBFF5
:1002A0000CD0400EE66EA00EE66E000EE66E5DEC23
:1002B00006F0E552E552E552166A05D06592656A88
:1002C00068D8FF0000D0E552E552E7CFD9FF120011
:1002D000F66A1750F76EF86AD890F736F836F736A0
:1002E000F836140EA66EF29E550EA76EAA0EA76ED5
:1002F000A682A6941200D9CFE6FFE1CFD9FFE6523D
:10030000DF6A000EE76E1818E8AE02D0183403D08A
:10031000E750D880185436E218505C6E5D6A5E6A09
:100320005CAE02D05D685E685C50195CF66E5D5034
:100330001A58F76E5E501B58F86EDF50EA6A1C0FB1
:10034000E96E000EEA22EF50F56E0D00DF2A180666
:10035000185009E0DF50EA6A1C0FE96E000EEA222D
:10036000EF50F56E01D0F5680C00DF2A240EA66E62
:10037000F29E550EA76EAA0EA76EA682185001E037
:100380001806BFD7A694186AE552E552E7CFD9FF01
:100390001200D9CFE6FFE1CFD9FFE652DF6AFF0EA8
:1003A000DF5C0AE2E868E85005E0E80600D000D02B
:1003B00000D0F9D7DF2AF3D7E552E552E7CFD9FFCE
:1003C0001200D9CFE6FFE1CFD9FFE652645032E107
:1003D0006296040100513C0BE842E8420D0828E116
:1003E000180E021923E1040E031920E1100E026F0A
:1003F000040E036FDF6ADF505C6E5D6A080E5C5CA2
:10040000000E5D5813E2DF50EA6A180FE96E040E21
:10041000EA22EF50E66EDF50EA6A100FE96E040E32
:10042000EA22E552E750EF6EDF2AE5D711D80AD06D
:1004300046D808D0040E645C03E162965CD802D012
:10044000000E01D0010EE552E552E7CFD9FF1200B0
:10045000D9CFE6FFE1CFD9FFE652040104BF046B18
:100460000C6A086A096A0A6A0B6A89EC03F0DF6A97
:10047000DF505C6E5D6A010E5C5C000E5D5819E237
:10048000095017E1F76ADF34FE0BF736F66E5E0EA1
:10049000F6260F0EF7220900F5CF5CF00800F5CF25
:1004A0005DF004D05DC0FAFF5C50F96EFBDFDF2A1F
:1004B000DFD7EDD8E552E552E7CFD9FF1200020EA3
:1004C000085C0EE1A7D80401180E026F040E036F3A
:1004D000080E016F00BD02D0C80E0BD0880E09D0E7
:1004E00014D90401080E016F100E026F040E036F81
:1004F0008C0E006F1200040E0E5C0AE112C438FF6D
:100500000F013851000802E2050E01D0030E0E6EF5
:1005100008040FE110D8020E0C5C03E10401840E04
:1005200006D0040104BD02D0C80E01D0880E046FAD
:10053000120085EF03F0D9CFE6FFE1CFD9FF020E1D
:10054000E126080E0A5C000E0B580DE20AC0DEFF21
:100550000BC0DDFF0C5002E1010E03D00C0406E1DC
:10056000020E0C6E03D0080EDE6EDD6A04010493E9
:100570000491010EDB500413DFCF05F4DE500A5E58
:10058000DD500B5A0001180EE26F040EE36F0FA24C
:100590001CD0D9CFE9FFDACFEAFFEE50ED1030E002
:1005A000E0C0F6FFE1C0F7FF0800F550E2C0E9FF48
:1005B000E3C0EAFFEF6EE22B000EE323E02BE12322
:1005C000DF06010EE6E2DB06E4D7D9CFE9FFDACF9A
:1005D000EAFFEE50ED1014E0E0C0E9FFE1C0EAFFF1
:1005E000EF50E2C0E9FFE3C0EAFFEF6EE22B000E3E
:1005F000E323E02BE123DF06010EE7E2DB06E5D78C
:10060000020EE15C02E2E16AE552E16EE552E7CFFB
:10061000D9FF1200D9CFE6FFE1CFD9FF020EE126C4
:10062000030E04010015E76E010EE7CFDBFF01C4E6
:10063000DFFFDE500A26DD500B220001180EE06FAE
:10064000040EE16FD9CFE9FFDACFEAFFEE50ED10EB
:1006500014E0E0C0E9FFE1C0EAFFEF50E2C0E9FFCB
:10066000E3C0EAFFEF6EE22B000EE323E02BE12371
:10067000DF06010EE7E2DB06E5D7020EE15C02E2EF
:10068000E16AE552E16EE552E7CFD9FF12006598C5
:1006900009500BE10401080E016F100E026F040EE9
:1006A000036F840E006F04011ED0040110AF1DD033
:1006B0000A50165D0B50175904E216C40AF017C40D
:1006C0000BF039DF010E086E0401080E016F100EE9
:1006D000026F040E036F800E006F0401180E066F88
:1006E000040E076FC80E046F1200020E086E04019C
:1006F000056BC80E046F0401080E016F180E026F1F
:10070000040E036FC80E006F1200086A0401046B28
:10071000120004011051600BE842E842E842E8424E
:10072000E842000901E012001151070A43E00B0AF8
:1007300041E0070A34E0010A24E00B0A20E0020A43
:100740001EE0030A1AE0080A10E0010A0CE00F0A92
:1007500008E0030A01E01200010E096E040E0E6E9D
:100760001200DBEF03F02BEF04F0010E096E000125
:10077000100EE06F000EE16F0ED04FEF04F090EF1F
:1007800004F0010E096E14510001E06FE16B110ECF
:10079000E027000EE1230F92010E0A6E1200010EF7
:1007A000096E1451EA6A110FE96E000EEA2212C4B2
:1007B000EFFF12001200800E0401105D4BE1135197
:1007C000030A2DE0010A0BE0030A43E1010E096E62
:1007D00000019E0EE06F0E0EE16F120E38D0010E7A
:1007E000096E1251F66EF76AD890F636F736540E47
:1007F000F6260F0EF7220900F5CFE0F00A00F5CF3C
:10080000E1F0020E0001F76AE025F66EE151F722F1
:100810000900F5CF0AF00A00F5CF0BF01AD0010E4F
:10082000096E1251F66EF76AD890F636F736580E02
:10083000F6260F0EF7220900F5CFE0F00A00F5CFFB
:10084000E1F0E0C0F6FFE1C0F7FF0800F5500A6EE6
:100850000B6A0F821200010E096E0F0EE66E270E54
:10086000E66E0F0EE66ECBEC05F0E552E552E55272
:10087000010EE66E110EE66E000EE66ECBEC05F094
:10088000E552E552E55212C410F00401125103E1A1
:10089000050E0E6E1200060E0E6E48EF06F00401F5
:1008A000186B196B040110511F0B020A0EE0030AAA
:1008B00009E0010A2AE1010E096E0FA026D0040109
:1008C000188323D0010E096E20D0010E096E145139
:1008D0000F0B080DF3505D6A000F5C6E040E5D2275
:1008E0001451800B01E0010E040DF35000015C2453
:1008F000E26F000E5D20E36FE2C0E9FFEA6EEF50A9
:10090000040B03E00401010E186F090408E1000163
:10091000180EE06F040EE16F0F92020E0A6E1200C5
:10092000040112050CE110511F0B000908E1010E32
:10093000096E030E115D02E10F8001D00F9012517C
:1009400034E110511F0B020830E114510F0B000964
:100950002CE0010E096E14510F0B080DF3505D6A67
:10096000000F5C6E040E5D221451800B01E0010E3D
:10097000040DF35000015C24E26F000E5D20E36F74
:10098000030E0401115D02E1840E03D014AF07D001
:10099000400EE2C0E9FFE3C0EAFFEF6E1200880EEE
:1009A000E2C0E9FFE3C0EAFFEF6E120065A60CD8D3
:1009B0000E0409E165BA07D0626A0F01366B368111
:1009C0003689020E0E6E1200656A0F01366B65865F
:1009D000010E0E6E1200656A0F01366B0E6A120070
:1009E000EBEF04F00E5001E112006250040B05E041
:1009F0000F013651040B01E083D865B2120062503A
:100A0000010B05E00F013651010B01E093D8625054
:100A1000100B05E00F013651100B01E01FD862509A
:100A2000200B05E00F013651200B01E071D8030EB9
:100A30000E5C01E212000D6A040E0D5C0EE26250C3
:100A4000080B0BE00F013651080B07E0E1EC01F059
:100A5000000901E162960D2AEFD71200D9CFE6FF17
:100A6000E1CFD9FF020EE12636CFDFFF0F01040EE2
:100A7000366F629865828C50040B01E0010E5C6E4B
:100A80008C50080B01E0010E5C10E76E010EE7CF01
:100A9000DBFF8C968C94A198A0880300A150100BCA
:100AA00005E1D050080B02E10300F8D7A098DF5011
:100AB0000F013613010EDB50E8B08C86E8A08C964F
:100AC000010EDB50E8B08C84E8A08C94D50E056E46
:100AD000020E066E05C05CF006C05DF00506000E55
:100AE000065A5C505D1002E00400F4D7020EE15C8F
:100AF00002E2E16AE552E16EE552E7CFD9FF12006A
:100B000065920F01369562A402D06294FCD7120060
:100B10000F0126A10DD0800E0401005D07E1840EB7
:100B20000401045D03E104018C0E006F0F012691A6
:100B3000629A1200636A626A0F019F0E376F0F019B
:100B40007B0E366F0F01386B0F0EE66E270EE66ECA
:100B50000F0EE66E20D8E552E552E5520F01160E53
:100B6000266F62A605D0629600D000D00000F9D7AB
:100B7000659885EC03F00401080E016F0401100E66
:100B8000026F040E036F04018C0E006F0F90106A49
:100B9000030E0E6E1200D9CFE6FFE1CFD9FFFD0E96
:100BA000DBCFE9FFFE0EDBCFEAFFFC0EDB5004E0FB
:100BB000EE6AFC0EDB06F9D7E552E7CFD9FF12004B
:100BC000040110511F0B010801E01200145101E053
:100BD0001200060E115D21E11351230A1DE0010AE6
:100BE0000DE0030A19E1020E096E100405E100018F
:100BF000C20EE06F0E0EE16F090E0CD0020E096EF0
:100C0000100405E10001370EE06F0F0EE16F1004D4
:100C100003E11D0E0A6E0B6A0F8204011051600B76
:100C2000E842E842E842E842E842010801E01200F6
:100C300011510B0A26E0080A19E0090A12E0080A15
:100C400009E00B0A05E0080A01E0120046EF06F091
:100C500047EF06F0020E096E0001000EE06F000E75
:100C60000BD0020E096E13C400F01200020E096EC2
:100C70000001010EE06F000EE16F0F92010E0A6E8F
:100C80001200020E096E12C401F0120012001200CE
:100C9000026A0F011E0E276F0401400E096F200E1D
:100CA0000A6F040E0B6F880E086F0401600E0E6F42
:100CB000040E0F6F400E0C6F1200D9CFE6FFE1CF8C
:100CC000D9FFE652FC0EDB50400805E2400EF36E01
:100CD000FC0EF3CFDBFFDF6AFC0EDB50DF5C19E2BA
:100CE000DF50E76EFD0EDBCFE9FFFE0EDBCFEAFF44
:100CF000E750E926000EEA22EF50E66EDF50EA6A7E
:100D0000600FE96E040EEA22E552E750EF6EDF2A2B
:100D1000E3D7FC0EDBCF0DF4400E04010C170C7D65
:100D2000880E0C13E552E552E7CFD9FF1200D9CF58
:100D3000E6FFE1CFD9FF026A040108BF2FD0FC0E05
:100D4000DBCF5CF00951D8805C5403E2FC0E09C48F
:100D5000DBFF026AFC0EDB50025C19E20250EA6A19
:100D6000200FE96E040EEA22EF50E66E0250E76EA5
:100D7000FD0EDBCFE9FFFE0EDBCFEAFFE750E926F1
:100D8000000EEA22E552E750EF6E022AE3D7040193
:100D9000400E096F0817087D880E08130250E552AF
:100DA000E7CFD9FF12001DEE00F02DEE00F0F86A3B
:100DB000F66A100EF76E0800F550FF0808E1010E04
:100DC000F66E100EF76E0800F550FF0806E080AED4
:100DD00002D000EF08F080AEFED701D812000DD887
:100DE000040034D837D8060E0E5C05E16550020BBE
:100DF00002E125EC00F0F4D71200600ED36E9B8C5C
:100E0000580E056E020E066E05C05CF006C05DF061
:100E10000506000E065A5C505D10F6E165A604D08A
:100E20006592656AC9EC01F00F01140E396F0E6A04
:100E30000F6A106A19EC00F0036A046A8C968C94AD
:100E4000959695940F01486B496B1200D6EC04F00F
:100E5000F2EF04F00350041004E1100E036E270EAD
:100E6000046E0306000E045A060E0E5C02E28C8627
:100E70008C94060E0E5C12E1035004100FE1000189
:100E8000075102E18C868C94030E075D02E18C967B
:100E90008C84072B0751030801E2076B1200120133
:100EA000000200000008D8043C000200010200011A
:100EB00009022900010100C03209040000020300F8
:100EC0000000092111010001221D000705810340D6
:100ED0000001070501034000010403090434034D28
:100EE000006900630072006F0063006800690070B1
:100EF00000200054006500630068006E006F006C05
:100F0000006F0067007900200049006E0063002E2A
:100F100000260348004900440020005500530042C9
:100F200000200042006F006F0074006C006F0061D1
:100F3000006400650072000600FF0901A1011901AB
:100F40002940150026FF00750895408100190129E8
:100F5000409100C0B00EB00ED90EDD0E110FC00BC7
:100F6000C00EF36E00EE00F00E0E01D81200EA6023
:100F700002D0EE6AFCD7F350E9601200EE6AFCD7AB
:06100000FAEF39F01200C6
:06100800CFEF25F01200FD
:0610180022EF08F01200B7
:10102A00020042740000990100006400000040744C
:10103A000000B70E000002000000D8CFE4FFE0CFA6
:10104A00E4FFE46EDACFE4FFE2CFDAFFE9CFE4FFB0
:10105A00EACFE4FFF3CFE4FFF4CFE4FFE652D9CFBF
:10106A00E6FFE1CFD9FF040EE126020EDB6A030E8A
:10107A00DB6A9EA27AD39E920401D45101E1A1D0E7
:10108A00030E526E2D50EA6A510FE96E010EEA22E2
:10109A00EF50525C30E12D50E96EEA6AD890E93699
:1010AA00EA36690EE926010EEA22EECF52F0EFCFB8
:1010BA0053F053C052F0536A5250D76E2D50E96E16
:1010CA00EA6AD890E936EA36690EE926010EEA227A
:1010DA00EECF52F0EFCF53F05250D66EF28AF2941E
:1010EA00D58E2D50EA6A510FE96E010EEA22040EDE
:1010FA00EF6E2D502F6E020E526E2E50EA6A510F6D
:10110A00E96E010EEA22EF50525C49E12E50E96E77
:10111A00EA6AD890E936EA36690EE926010EEA2229
:10112A00EE50ED1009E12E50EA6A510FE96E010EF8
:10113A00EA22010EEF6E33D0080E2E5C0CE2070E87
:10114A002E14526E010E525204E0E846FE0B52066D
:10115A00FCE189121AD0100E2E5C0CE2070E2E1436
:10116A00526E010E525204E0E846FE0B5206FCE1B2
:10117A008A120BD0070E2E14526E010E525204E040
:10118A00E846FE0B5206FCE18B122E50EA6A510F1A
:10119A00E96E010EEA22030EEF6E2E502D6E2E2AF4
:1011AA00060E2E5C02E1080E04D0130E2E5C03E13B
:1011BA00160E2E6E59D1180E2E5C01E055D12E6AEC
:1011CA0053D10E01005101E14FD10E01012B0E0145
:1011DA00AC510E01015D01E247D1016B0E01AA512A
:1011EA00EA6A320FE96E0E0EEA22EF500E01EA6A3F
:1011FA00AD25E96EAE51EA22EF6A79907B6A7A6A86
:10120A000E01AA2B0E01AB510E01AA5D01E3AA6BD6
:10121A00AA51E96EEA6AD890E936EA36020EE92658
:10122A000E0EEA22EE50ED1001E11ED1AA51E96E2E
:10123A00EA6AD890E936EA364A0EE9260E0EEA221A
:10124A00EECF52F0EFCF53F0AA51E96EEA6AD89086
:10125A00E936EA36020EE9260E0EEA22EECF54F0FD
:10126A00EFCF55F05450521802E15550531801E18E
:10127A00BDD0AA51E96EEA6AD890E936EA364A0E32
:10128A00E9260E0EEA22EECF54F0EFCF55F0AA511E
:10129A00E96EEA6AD890E936EA36020EE9260E0EB7
:1012AA00EA22EE50545C526EEE505558536E020EBE
:1012BA0052C0DBFF030E53C0DBFF020EDBCF52F03E
:1012CA00030EDBCF53F053343BE252500008000EBA
:1012DA00535436E2020EDBCF52F0030EDBCF53F04B
:1012EA00AA51E96EEA6AD890E936EA367A0EE92610
:1012FA000E0EEA22EECF54F0EFCF55F05250545C66
:10130A005350555857E2AA51E96EEA6AD890E9361D
:10131A00EA367A0EE9260E0EEA22EECF52F0EFCF27
:10132A0053F0AA51E96EEA6AD890E936EA36020E13
:10133A00E9260E0EEA225250EE265350ED2256D0DE
:10134A00020EDBCF52F0030EDBCF53F0526C531E6A
:10135A00000E5322AA51E96EEA6AD890E936EA36B3
:10136A007A0EE9260E0EEA22EECF54F0EFCF55F0B0
:10137A005250545C535055581DE2AA51E96EEA6A1C
:10138A00D890E936EA367A0EE9260E0EEA22EECF30
:10139A0052F0EFCF53F0AA51E96EEA6AD890E936D3
:1013AA00EA36020EE9260E0EEA225250EE5E53503B
:1013BA00ED5A1CD0AA51E96EEA6AD890E936EA36A3
:1013CA004A0EE9260E0EEA22EECF52F0EFCF53F084
:1013DA00AA51E96EEA6AD890E936EA36020EE92697
:1013EA000E0EEA2252C0EEFF53C0EDFFAA51EA6A7E
:1013FA00320FE96E0E0EEA22EF500E01EA6AAD25AF
:10140A00E96EAE51EA22120EEF6EF29E0E01AA5159
:10141A00E96EEA6AD890E936EA36020EE9260E0E35
:10142A00EA22EECF52F0EFCF53F053C052F0536A94
:10143A005250B66EAA51E96EEA6AD890E936EA368F
:10144A00020EE9260E0EEA22EECF52F0EFCF53F04B
:10145A005250B56EF00EB4140009B46EF00EB41406
:10146A000909B46E7980F28E000ED8802154000EDC
:10147A0022542EE2302A000E31222150305C2250B2
:10148A00315826E3306A316A030E255C1FE2235085
:10149A00EA6A480FE96E010EEA2280CFEFFF235075
:1014AA00EA6A4B0FE96E010EEA2281CFEFFF235061
:1014BA00EA6A4E0FE96E010EEA2282CFEFFF232A73
:1014CA00030E235C01E3236A252A02D0216A226AD9
:1014DA00000ED8802654000E275419E22B5000081B
:1014EA0016E2322A000E33222650325C2750335835
:1014FA000EE3326A336A030E2A5C07E2282A030ED5
:10150A00285C01E3286A2A2A02D0266A276A2B5015
:10151A0000080AE2346A3450040DF328C26E9E9C15
:10152A009F9C9D8CC280C2820101995101E11DD10B
:10153A00DE6ADD6ADECF52F0DDCF53F0040E525C74
:10154A00000E535801E311D1DECFE9FFDDCFEAFFE8
:10155A00010ED890E936EA36E806FBE19A0EE9264A
:10156A00010EEA22EE50ED1001E1D3D0DECFE9FF01
:10157A00DDCFEAFF010ED890E936EA36E806FBE14C
:10158A00AA0EE926010EEA22EE50ED1026E1D9CF85
:10159A00E9FFDACFEAFFEE50ED1001E18180D9CF01
:1015AA00E9FFDACFEAFF010EEE1803E1ED5001E19F
:1015BA008182D9CFE9FFDACFEAFF020EEE1803E102
:1015CA00ED5001E18184D9CFE9FFDACFEAFF030EBA
:1015DA00EE1803E1ED5001E18186DECFE9FFDDCFB0
:1015EA00EAFF010ED890E936EA36E806FBE1AA0ED0
:1015FA00E926010EEA22EECF52F0EFCF53F0DECF0A
:10160A00E9FFDDCFEAFF010ED890E936EA36E806AF
:10161A00FBE19A0EE926010EEA22EECF54F0EFCF53
:10162A0055F05450521829E15550531826E1D9CF94
:10163A00E9FFDACFEAFFEE50ED1001E18190D9CF50
:10164A00E9FFDACFEAFF010EEE1803E1ED5001E1FE
:10165A008192D9CFE9FFDACFEAFF020EEE1803E151
:10166A00ED5001E18194D9CFE9FFDACFEAFF030E09
:10167A00EE1803E1ED5001E18196DECFE9FFDDCFFF
:10168A00EAFF010ED890E936EA36E806FBE1AA0E2F
:10169A00E926010EEA22EE2A000EEF22DECFE9FF4A
:1016AA00DDCFEAFF010ED890E936EA36E806FBE11B
:1016BA00AA0EE926010EEA22EECF52F0EFCF53F03E
:1016CA00DECFE9FFDDCFEAFF010ED890E936EA3630
:1016DA00E806FBE1A20EE926010EEA22EECF54F05B
:1016EA00EFCF55F0545052183AE15550531837E19C
:1016FA00DECFE9FFDDCFEAFF010ED890E936EA3600
:10170A00E806FBE1AA0EE926010EEA22EE6AED6A74
:10171A0026D0D9CFE9FFDACFEAFFEE50ED1001E18A
:10172A008190D9CFE9FFDACFEAFF010EEE1803E183
:10173A00ED5001E18192D9CFE9FFDACFEAFF020E3B
:10174A00EE1803E1ED5001E18194D9CFE9FFDACF38
:10175A00EAFF030EEE1803E1ED5001E18196DF2A5C
:10176A00010E01E2E7D6DB2AE5D69EAC2CD09E9C80
:10177A00C450566E576E566AC35000015610546EC6
:10178A0057C055F03450060DF3CF52F0F4CF53F052
:10179A00000E5226010E53222850020D5250F324F5
:1017AA00E96E5350F420EA6E54C0EEFF55C0EDFFC7
:1017BA00342A2B50345C02E39D9C05D03450040D2E
:1017CA00F328C26EC282F2A442D0D59EF294F29A53
:1017DA00040E526E2F50EA6A510FE96E010EEA2288
:1017EA00EF50525C34E1080E2F5C0DE2070E2F1405
:1017FA00526E010E525204E0E846FE0B5206FCE11C
:10180A00E81C89161CD0100E2F5C0DE2070E2F144F
:10181A00526E010E525204E0E846FE0B5206FCE1FB
:10182A00E81C8A160CD0070E2F14526E010E525263
:10183A0004E0E846FE0B5206FCE1E81C8B162F502A
:10184A00EA6A510FE96E010EEA22020EEF6E040EE9
:10185A00E15C02E2E16AE552E16EE552E7CFD9FFC7
:10186A00E552E5CFF4FFE5CFF3FFE5CFEAFFE5CF99
:10187A00E9FFE5CFDAFFE550E5CFE0FFE5CFD8FF96
:10188A001000D9CFE6FFE1CFD9FF020EE126896A1F
:10189A0092682B6A8A6A93688B6A94688C968C948D
:1018AA0095969594928E0401010ED36F0E01B76935
:1018BA00B869296A286A2A6A246A236A256A216A0F
:1018CA00226A266A276A306A316A326A336A346A55
:1018DA00CA82CA80CA9CCA9ACA88CA96FA0ECB6EAB
:1018EA00DF6ADFCF49F00C0EE76E4918E8AE02D086
:1018FA00E73402D0E750495C36E2010EDB6ADBCFFF
:10190A0049F0030EE76E4918E8AE02D0E73402D078
:10191A00E750495C26E2DFCF49F04A6A49BE4A6885
:10192A00060E4A02F3CF4AF04902F3CF49F0F450C7
:10193A004A26000E4926010E4A22010EDBCF4BF041
:10194A004C6A4BBE4C68D8904B364C3649504B24A7
:10195A00E96E4A504C20EA6EEE6AED6A010EDB2A05
:10196A00CED7DF2ABED70401CD6BCE6BCB6BCC6B47
:10197A00CF6BD06BD16BD26B2D6A2E6A2F6ADF6A5E
:10198A00DFCF49F0180EE76E4918E8AE02D0E73407
:10199A0002D0E750495C1BE2DFCFE9FFEA6AE9BE01
:1019AA00EA68D890E936EA36690EE926010EEA2293
:1019BA00EE6AED6ADFCFE9FFEA6AE9BEEA68510E2C
:1019CA00E926010EEA22010EEF6EDF2AD9D7D58663
:1019DA00D59AD59CF294F29AF194D08ECA949D82AB
:1019EA009F9253EC27F0A0EC34F0F28EF28CCA846A
:1019FA00020EE15C02E2E16AE552E16EE552E7CFEE
:101A0A00D9FF1200D9CFE6FFE1CFD9FF050EE126B3
:101A1A00020EDB6A030EDB6A040EDB6AD5EC1CF0ED
:101A2A002550000809E2D4EC13F0242A030E245CA2
:101A3A0001E1246A2506F4D72A50000809E204ECD9
:101A4A0014F0292A030E295C01E1296A2A06F4D72F
:101A5A00200E0501E76EA819E8AE02D0E73402D0DD
:101A6A00E750A85D01E2B7D16550020B01E0B3D19E
:101A7A00400EE66E400EE66E020EE66E03EC33F0A2
:101A8A00E552E552E552E76E030EE7CFDBFFDB5086
:101A9A00000801E324D1040EDB6A030EDB50F36E67
:101AAA00040EDBCFF4FFF350F45C01E318D1040E0B
:101ABA00DB50EA6A400FE96E020EEA22EFCFDFFF3F
:101ACA000101F65141E10D0E496EDF50495C05E016
:101ADA000A0E4A6EDF504A5C37E1010EF66F0401C6
:101AEA00CD51EA6A000FE96E030EEA220D0EEF6E7F
:101AFA00CD2B010EDB6ACD51F36E010EDBCFF4FF65
:101B0A00F350F45C1CE2010EDBCFE9FFEA6AE9BE9E
:101B1A00EA68000EE926030EEA22EF50E66E010E8D
:101B2A00DBCFE9FFEA6AE9BEEA68B20EE926010EEE
:101B3A00EA22E552E750EF6E010EDB2ADCD7D5D94F
:101B4A000401CD6BCE6BBBD01B0EDF5C09E1F251F9
:101B5A0007E1010EF26F1B0EF36FF46BF56BAFD05A
:101B6A00F2050BE15B0EDF5C08E11B0EF35D05E19C
:101B7A00F45103E15B0EF46FA2D0F20566E1410E67
:101B8A00DF5C63E11B0EF35D60E15B0EF45D5DE11A
:101B9A00F36BF46BF56BF26B010EDB6ADBCFE9FFDB
:101BAA00EA6AE9BEEA68000EE926030EEA22EF5065
:101BBA000D081CE0010EDBCFE9FFEA6AE9BEEA681C
:101BCA00B20EE926010EEA22EF50E66E010EDBCFD5
:101BDA00E9FFEA6AE9BEEA68000EE926030EEA228C
:101BEA00E552E750EF6E010EDB2AD8D7010EDBCFA4
:101BFA00CDF40401CD51EA6A000FE96E030EEA2220
:101C0A00EF6AF90E496E6D0E4A6E4B6A49C0E6FFDD
:101C1A00E66E4BC0E6FF31EC38F0E552E552E5528C
:101C2A00000EE66E030EE66EF60E496E6D0E4A6EF5
:101C3A004B6A49C0E6FFE66E4BC0E6FF31EC38F06E
:101C4A004C6E050EE15E4C503AD0080EDF5C1CE18A
:101C5A000401CD51000818E2CD07CD51EA6A000F00
:101C6A00E96E030EEA22EF6AF30E496E6D0E4A6EB2
:101C7A004B6A49C0E6FFE66E4BC0E6FF31EC38F02E
:101C8A00E552E552E5521BD00D0EDF5C18E00A0E54
:101C9A00DF5C15E0200EDF5C12E30101F36BF46BED
:101CAA00F56BF26B0401CD51EA6A000FE96E030E7F
:101CBA00EA22DFCFEFFF0101F66B0401CD2B04010D
:101CCA00CD51496E4A6A000E491806E1010E4A18BA
:101CDA0003E12C86CD6BCE6B040EDB2ADED62C50AC
:101CEA0001E178D02CA00FD0ED0E496E6D0E4A6E30
:101CFA004B6A49C0E6FFE66E4BC0E6FF31EC38F0AE
:101D0A00E552E552E5522CA20FD0CE0E496E6D0E69
:101D1A004A6E4B6A49C0E6FFE66E4BC0E6FF31ECFD
:101D2A0038F0E552E552E5522CA40FD0B20E496EB6
:101D3A006D0E4A6E4B6A49C0E6FFE66E4BC0E6FF7F
:101D4A0031EC38F0E552E552E5522CA60FD0960E4A
:101D5A00496E6D0E4A6E4B6A49C0E6FFE66E4BC08D
:101D6A00E6FF31EC38F0E552E552E5522CA80FD0E7
:101D7A00770E496E6D0E4A6E4B6A49C0E6FFE66EF3
:101D8A004BC0E6FF31EC38F0E552E552E5522CAC97
:101D9A000FD0560E496E6D0E4A6E4B6A49C0E6FF69
:101DAA00E66E4BC0E6FF31EC38F0E552E552E552FB
:101DBA002CAE0FD03D0E496E6D0E4A6E4B6A49C06D
:101DCA00E6FFE66E4BC0E6FF31EC38F0E552E5522D
:101DDA00E5522C6A3FD8050EE15C02E2E16AE5525F
:101DEA00E16EE552E7CFD9FF1200D9CFE6FFE1CF86
:101DFA00D9FFE652CBC4DFFFDF2A400E496EDF501F
:101E0A00495C01E1DF6A0401CC51DF5C01E122D8BF
:101E1A000401CB51EA6A000FE96E020EEA22FE0EB5
:101E2A00DBCFEFFFCB2B400ECB5D01E1CB6BCC516F
:101E3A00CB5D01E12C84FE0EDBCF49F04A6A49BE34
:101E4A004A6849C0F3FF4AC0F4FFE552E552E7CFBA
:101E5A00D9FF1200D9CFE6FFE1CFD9FFE65204013C
:101E6A00CB51CC5D3DE00501905105E0FBEC33F030
:101E7A00C6EC1DF0F8D70401CC51D880CB5517E237
:101E8A00CC51CB5DDF6EDFCFE6FFCC514A6A000F43
:101E9A00496E020E4A2249C0E6FF4AC0E6FF63ECD9
:101EAA0033F0E552E552E552CBC4CCF417D0400EDC
:101EBA00D880CC55DF6EDFCFE6FFCC514A6A000FDF
:101ECA00496E020E4A2249C0E6FF4AC0E6FF63ECA9
:101EDA0033F0E552E552E5520401CC6BFBEC33F0EA
:101EEA00E552E552E7CFD9FF1200D9CFE6FFE1CF9D
:101EFA00D9FF040EE126DE6ADD6A020EDB6A030EF2
:101F0A00DB6A0401CE51EA6A000FE96E030EEA2287
:101F1A00EF50E66EE66A8AEC39F0E552E552020EB7
:101F2A00F3CFDBFF0401CE2BCE51496E4A6A000E75
:101F3A00491804E1010E4A1801E1CE6B020EDB508A
:101F4A00DE6EDD6ACE51EA6A000FE96E030EEA22FE
:101F5A00EF502C0836E0CE51EA6A000FE96E030E04
:101F6A00EA22EF500D082DE0CE51EA6A000FE96E21
:101F7A00030EEA22EF50E66EE66A8AEC39F0E55281
:101F8A00E552030EF3CFDBFF0401CE2BCE51496E8F
:101F9A004A6A000E491804E1010E4A1801E1CE6BA3
:101FAA00020EDBCF4BF04BC04CF04B6A030EDB50FA
:101FBA0000014B24496E000E4C204A6E49C0DEFFD8
:101FCA00DD6E000EDFCF3DF0010EDBCF3EF0320EAC
:101FDA003D1802E1530E3E1801E1AAD14B0E3D18FD
:101FEA0002E1430E3E1801E1A0D14C0E3D1802E178
:101FFA00420E3E1801E196D1440E3D1802E14E0E02
:10200A003E1801E18CD1490E3D1802E14E0E3E18F0
:10201A0001E182D1420E3D1802E1510E3E1801E162
:10202A0078D14C0E3D1802E1510E3E1801E16ED1F5
:10203A004C0E3D1802E1530E3E1801E164D14E0EDA
:10204A003D1802E1510E3E1801E15AD14E0E3D18DB
:10205A0002E1530E3E1801E150D1430E3D1802E150
:10206A00530E3E1801E146D14D0E3D1802E1450ED0
:10207A003E1801E13CD1500E3D1802E1510E3E18C6
:10208A0001E132D1500E3D1802E1540E3E1801E131
:10209A0028D1500E3D1802E1530E3E1801E11ED11F
:1020AA004D0E3D1802E1530E3E1801E114D1470EC0
:1020BA003D1802E1500E3E1801E10AD1430E3D18C7
:1020CA0002E1500E3E1801E100D1490E3D1802E12D
:1020DA00430E3E1801E1F6D0490E3D1802E1520EB8
:1020EA003E1801E1ECD0490E3D1802E1530E3E18AC
:1020FA0001E1E2D0530E3D1802E1430E3E1801E120
:10210A00D8D0530E3D1802E1520E3E1801E1CED04E
:10211A00530E3D1802E1530E3E1801E1C4D0530E8E
:10212A003D1802E1420E3E1801E1BAD0430E3D18B5
:10213A0002E1420E3E1801E1B0D0430E3D1802E121
:10214A00520E3E1801E1A6D04F0E3D1802E1420E92
:10215A003E1801E19CD0570E3D1802E14D0E3E1883
:10216A0001E193D0520E3D1802E14D0E3E1801E1F5
:10217A008AD0440E3D1802E1500E3E1801E181D08A
:10218A004F0E3D1802E1500E3E1801E177D0490E7C
:10219A003D1802E1500E3E186EE0580E3D1802E15D
:1021AA00540E3E1865E0540E3D1801E13E505EE0C3
:1021BA00410E3D1801E13E5057E0560E3D1801E12F
:1021CA003E5050E0490E3D1801E13E5049E04F0EA5
:1021DA003D1801E13E5042E0550E3D1802E1430E22
:1021EA003E183AE0580E3D1802E1430E3E1831E01F
:1021FA00430E3D1801E13E502AE0520E3D1801E11E
:10220A003E5023E0580E3D1802E1520E3E181AE0E5
:10221A00030EDB5001E08FD0020EDBCFE6FFE66A49
:10222A00DBCFE6FFE66A1A0E496E6D0E4A6E4B6AFE
:10223A0049C0E6FFE66E4BC0E6FF31EC38F04C6E63
:10224A00070E97D04AEC17F096D0CBD894D060D925
:10225A0092D04CEC17F08FD0C8D88DD017DA8BD02B
:10226A009EDA89D0BCDA87D0CADA85D006D983D07B
:10227A0048EC17F080D0C7EC15F07DD064EC16F06E
:10228A007AD09ADB78D056DB76D016DB74D000ECA5
:10229A0018F071D04EEC17F06ED0FEEC17F06BD040
:1022AA0002EC18F068D004EC18F065D006EC18F0CF
:1022BA0062D008EC18F05FD00AEC18F05CD00CEC95
:1022CA0018F059D00EEC18F056D010EC18F053D084
:1022DA00A1EC18F050D0DCEC28F04DD0CEEC2AF06E
:1022EA004AD096EC2AF047D07BEC2AF044D034EC62
:1022FA002BF041D0A5EC27F03ED0DDEC2BF03BD003
:10230A000DEC2CF038D027EC2CF035D039EC2CF031
:10231A0032D054EC2CF02FD0BFEC2BF02CD0D0ECD8
:10232A002BF029D0C6EC18F026D0CBEC18F023D02D
:10233A002AEC35F020D0030EDBCFE6FFE66A020E68
:10234A00DBCFE6FFE66A030EDBCFE6FFE66A020EA4
:10235A00DBCFE6FFE66AF20E496E6C0E4A6E4B6AF6
:10236A0049C0E6FFE66E4BC0E6FF31EC38F04C6E32
:10237A000B0EE15E4C500401CE51EA6A000FE96E81
:10238A00030EEA22EF500D080DE02C500BE1520E1D
:10239A00496E4A6ADF50491803E1DE52DD504A1895
:1023AA0001E02C8ECDC4CEF4040EE15C02E2E16AB7
:1023BA00E552E16EE552E7CFD9FF12000401D3518D
:1023CA000FE0A80E496E730E4A6E4B6A49C0E6FFCB
:1023DA00E66E4BC0E6FF31EC38F0E552E552E552C5
:1023EA00120046EC0CF0E3EF11F0D9CFE6FFE1CF93
:1023FA00D9FF030EE126E66AD9CFE6FFDACFE6FF78
:10240A00010EE66E05EC1AF0E552E552E552E55288
:10241A00E66AD950010FE66E000EDA20E66E020E69
:10242A00E66E05EC1AF0E552E552E552E5522C50FB
:10243A001AE1DF0417E1D950010FE96EDACFEAFF9A
:10244A00EE50ED100AE0010E496E4A6ADB50491857
:10245A0008E1020EDB504A1804E1010EDBCFD3F487
:10246A0001D02C8CABDF030EE15C02E2E16AE5529B
:10247A00E16EE552E7CFD9FF1200D9CFE6FFE1CFEF
:10248A00D9FF030EE126020EDB6AE66A1F0EE66E2C
:10249A00000EE66E030EE66E05EC1AF0E552E55202
:1024AA00E552E552E66AD950020FE66E000EDA20CE
:1024BA00E66E010EE66E05EC1AF0E552E552E552BB
:1024CA00E5522C501BE1020EDB500CE11F5020108C
:1024DA0003E1216A226A11D0CA841FC021F020C0F8
:1024EA0022F00BD01F50201003E1266A276A05D07C
:1024FA00CA841FC026F020C027F060DF030EE15C0B
:10250A0002E2E16AE552E16EE552E7CFD9FF120035
:10251A00D9CFE6FFE1CFD9FF0A0EE126E66AD9CF85
:10252A00E6FFDACFE6FF010EE66E05EC1AF0E55299
:10253A00E552E552E552E66AD950010FE66E000E01
:10254A00DA20E66E010EE66E05EC1AF0E552E55267
:10255A00E552E552E66AD950020FE66E000EDA201D
:10256A00E66E010EE66E05EC1AF0E552E552E5520A
:10257A00E552E66AD950040FE66E000EDA20E66EDE
:10258A00010EE66E05EC1AF0E552E552E552E55207
:10259A00E66AD950050FE66E000EDA20E66E010EE5
:1025AA00E66E05EC1AF0E552E552E552E552E66AA6
:1025BA00D950060FE66E000EDA20E66E010EE66EC0
:1025CA0005EC1AF0E552E552E552E552E66AD950B1
:1025DA00070FE66E000EDA20E66E010EE66E05ECD7
:1025EA001AF0E552E552E552E552E66AD950080F6B
:1025FA00E66E000EDA20E66E010EE66E05EC1AF0C3
:10260A00E552E552E552E552E66AD950090FE66EFF
:10261A00000EDA20E66E010EE66E05EC1AF0E552BF
:10262A00E552E552E552E66AD950030FE66E000E0E
:10263A00DA20E66E010EE66E05EC1AF0E552E55276
:10264A00E552E5522C5018E1DF50926E010EDB5034
:10265A00936E020EDB50946E040EDB50956E050EDF
:10266A00DB50966E030EDB500C0805E20C0EF36E7F
:10267A00030EF3CFDBFFA2DE0A0EE15C02E2E16A9F
:10268A00E552E16EE552E7CFD9FF1200D9CFE6FF56
:10269A00E1CFD9FF020EE126E66AD9CFE6FFDACF0B
:1026AA00E6FF010EE66E05EC1AF0E552E552E55238
:1026BA00E552E76E010EE7CFDBFF2C5066E1010E13
:1026CA00DB5002E1DF50896E010EE66ED9CFE6FFDC
:1026DA00DACFE6FFE66E05EC1AF0E552E552E5526E
:1026EA00E552E76E010EE7CFDBFF2C504EE1010EFB
:1026FA00DB5002E1DF508A6E010EE66ED9CFE6FFAB
:10270A00DACFE6FFE66E05EC1AF0E552E552E5523D
:10271A00E552E76E010EE7CFDBFF2C5036E1010EE2
:10272A00DB5002E1DF508B6E010EE66ED9CFE6FF79
:10273A00DACFE6FFE66E05EC1AF0E552E552E5520D
:10274A00E552E76E010EE7CFDBFF2C501EE1010ECA
:10275A00DB5002E1DF508C6E010EE66ED9CFE6FF48
:10276A00DACFE6FFE66E05EC1AF0E552E552E552DD
:10277A00E552E76E010EE7CFDBFF2C5006E1010EB2
:10278A00DB5002E1DF508D6E19DE020EE15C02E2DF
:10279A00E16AE552E16EE552E7CFD9FF12008450B3
:1027AA00E66EE66A8350E66EE66A8250E66EE66A8E
:1027BA008150E66EE66A8050E66EE66AD50E496E8C
:1027CA006C0E4A6E4B6A49C0E6FFE66E4BC0E6FFE6
:1027DA0031EC38F04C6E0D0EE15E4C501200B00E2A
:1027EA00496E730E4A6E4B6A49C0E6FFE66E4BC0ED
:1027FA00E6FF31EC38F0E552E552E5521200D9CF46
:10280A00E6FFE1CFD9FFE652DF6AD30E496E6C0EBE
:10281A004A6E4B6A49C0E6FFE66E4BC0E6FF31ECF2
:10282A0038F0E552E552E552DF6A2B50DF5C30E2C0
:10283A00DFCF49F04A6A49BE4A68060E4A02F3CF18
:10284A004AF04902F3CF49F0F4504A26000E4926CD
:10285A00010E4A222950020D4950F324E96E4A50CA
:10286A00F420EA6EEECFE6FFEFCFE6FFCD0E4B6E19
:10287A006C0E4C6E4D6A4BC0E6FFE66E4DC0E6FF2D
:10288A0031EC38F04E6E050EE15E4E50DF2ACDD7A0
:10289A00AD0E496E730E4A6E4B6A49C0E6FFE66E8C
:1028AA004BC0E6FF31EC38F0E552E552E552E5520D
:1028BA00E552E7CFD9FF1200D9CFE6FFE1CFD9FF22
:1028CA00030EE126E66AD9CFE6FFDACFE6FFE66E27
:1028DA0005EC1AF0E552E552E552E552E66AD9509E
:1028EA00020FE66E000EDA20E66E010EE66E05ECC9
:1028FA001AF0E552E552E552E5522C5011E1DECFCD
:10290A0049F0DDCF4AF0000E495C100E4A5807E242
:10291A00DECFE9FFDDCFEAFF020EDBCFEFFF4EDDB0
:10292A00030EE15C02E2E16AE552E16EE552E7CFAD
:10293A00D9FF1200D9CFE6FFE1CFD9FF030EE12676
:10294A00E66AD9CFE6FFDACFE6FFE66E05EC1AF0C3
:10295A00E552E552E552E5522C5024E1DECF49F02A
:10296A00DDCF4AF0000E495C100E4A5807E2DECF6E
:10297A00E9FFDDCFEAFF020EEFCFDBFF020EDBCF6E
:10298A00E6FFE66AC30E496E6C0E4A6E4B6A49C090
:10299A00E6FFE66E4BC0E6FF31EC38F04C6E050EF2
:1029AA00E15E4C50030EE15C02E2E16AE552E16E3F
:1029BA00E552E7CFD9FF1200D9CFE6FFE1CFD9FF21
:1029CA00030EE126E66AD9CFE6FFDACFE6FF050E67
:1029DA00E66E05EC1AF0E552E552E552E552E66A72
:1029EA00D950010FE66E000EDA20E66E010EE66E91
:1029FA0005EC1AF0E552E552E552E552E66AD9507D
:102A0A00020FE66E000EDA20E66E010EE66E05ECA7
:102A1A001AF0E552E552E552E5522C5001E0A8D0F1
:102A2A00020EDB50010801E2A0D0010EDB500708BC
:102A3A0001E29BD0410E496EDF50495C1AE1020E59
:102A4A00DB500CE1010EF36EDB5004E0D890F33654
:102A5A00E806FCE1F350F31C921689D0010EF36EDE
:102A6A00DB5004E0D890F336E806FCE1F35092120A
:102A7A007ED0420E496EDF50495C1AE1020EDB50ED
:102A8A000CE1010EF36EDB5004E0D890F336E80651
:102A9A00FCE1F350F31C93166AD0010EF36EDB507F
:102AAA0004E0D890F336E806FCE1F35093125FD0C5
:102ABA00430E496EDF50495C1AE1020EDB500CE10D
:102ACA00010EF36EDB5004E0D890F336E806FCE121
:102ADA00F350F31C94164BD0010EF36EDB5004E056
:102AEA00D890F336E806FCE1F350941240D0440E35
:102AFA00496EDF50495C1AE1020EDB500CE1010E0F
:102B0A00F36EDB5004E0D890F336E806FCE1F350AC
:102B1A00F31C95162CD0010EF36EDB5004E0D8900E
:102B2A00F336E806FCE1F350951221D0450E496EC2
:102B3A00DF50495C1AE1020EDB500CE1010EF36E24
:102B4A00DB5004E0D890F336E806FCE1F350F31CBE
:102B5A0096160DD0010EF36EDB5004E0D890F336D2
:102B6A00E806FCE1F350961202D02C8C01D026DC48
:102B7A00030EE15C02E2E16AE552E16EE552E7CF5B
:102B8A00D9FF1200D9CFE6FFE1CFD9FF030EE12624
:102B9A00020EDB6AE66AD9CFE6FFDACFE6FF050E58
:102BAA00E66E05EC1AF0E552E552E552E552E66AA0
:102BBA00D950010FE66E000EDA20E66E010EE66EBF
:102BCA0005EC1AF0E552E552E552E5522C506DE15A
:102BDA00010EDB50070854E3410E496EDF50495C91
:102BEA000BE1010EF36EDB5004E0D890F336E806F1
:102BFA00FCE1F35080143FD0420E496EDF50495C2D
:102C0A000BE1010EF36EDB5004E0D890F336E806D0
:102C1A00FCE1F35081142FD0430E496EDF50495C1A
:102C2A000BE1010EF36EDB5004E0D890F336E806B0
:102C3A00FCE1F35082141FD0440E496EDF50495C08
:102C4A000BE1010EF36EDB5004E0D890F336E80690
:102C5A00FCE1F35083140FD0450E496EDF50495CF6
:102C6A000FE1010EF36EDB5004E0D890F336E8066C
:102C7A00FCE1F3508414E76E020EE7CFDBFF02D0CB
:102C8A002C8C13D0DBCFE6FFE66ABA0E496E6C0EC7
:102C9A004A6E4B6A49C0E6FFE66E4BC0E6FF31EC6E
:102CAA0038F04C6E050EE15E4C50030EE15C02E218
:102CBA00E16AE552E16EE552E7CFD9FF1200D9CFBA
:102CCA00E6FFE1CFD9FF030EE126E66AD9CFE6FF98
:102CDA00DACFE6FF050EE66E93DBE552E552E552E2
:102CEA00E552E66AD950010FE66E000EDA20E66E6A
:102CFA00010EE66E85DBE552E552E552E552E66ADB
:102D0A00D950020FE66E000EDA20E66E010EE66E6C
:102D1A0077DBE552E552E552E5522C5001E0A9D0A5
:102D2A00020EDB50010801E2A0D0010EDB500708B9
:102D3A0001E29BD0410E496EDF50495C1AE1020E56
:102D4A00DB500CE1010EF36EDB5004E0D890F33651
:102D5A00E806FCE1F350F31C891689D0010EF36EE4
:102D6A00DB5004E0D890F336E806FCE1F350891210
:102D7A007ED0420E496EDF50495C1AE1020EDB50EA
:102D8A000CE1010EF36EDB5004E0D890F336E8064E
:102D9A00FCE1F350F31C8A166AD0010EF36EDB5085
:102DAA0004E0D890F336E806FCE1F3508A125FD0CB
:102DBA00430E496EDF50495C1AE1020EDB500CE10A
:102DCA00010EF36EDB5004E0D890F336E806FCE11E
:102DDA00F350F31C8B164BD0010EF36EDB5004E05C
:102DEA00D890F336E806FCE1F3508B1240D0440E3B
:102DFA00496EDF50495C1AE1020EDB500CE1010E0C
:102E0A00F36EDB5004E0D890F336E806FCE1F350A9
:102E1A00F31C8C162CD0010EF36EDB5004E0D89014
:102E2A00F336E806FCE1F3508C1221D0450E496EC8
:102E3A00DF50495C1AE1020EDB500CE1010EF36E21
:102E4A00DB5004E0D890F336E806FCE1F350F31CBB
:102E5A008D160DD0010EF36EDB5004E0D890F336D8
:102E6A00E806FCE1F3508D1202D02C8C02D0E3EC80
:102E7A0011F0030EE15C02E2E16AE552E16EE5520D
:102E8A00E7CFD9FF1200E3EF11F0E3EF11F0E3EF20
:102E9A0011F0D9CFE6FFE1CFD9FF040EE126E66AA9
:102EAA00D9CFE6FFDACFE6FF050EE66EA9DAE552DC
:102EBA00E552E552E552E66AD950010FE66E000E78
:102ECA00DA20E66E010EE66E9BDAE552E552E5522D
:102EDA00E552E66AD950020FE66E000EDA20E66E77
:102EEA00030EE66E8DDAE552E552E552E5522C50B4
:102EFA0076E1D950020FE96EDACFEAFF720ED88076
:102F0A00EE542E0EED5441E3D950020FE96EDACF9A
:102F1A00EAFFEE50ED101FE04C684D684E6A2D0E28
:102F2A00E76E020EDBCF4FF0030EDBCF50F0E75017
:102F3A004F26000E5022516A4F504C5C496E505039
:102F4A004D584A6E51504E584B6E020E49C0DBFF27
:102F5A00030E4AC0DBFF010EDB50070816E3410EE1
:102F6A00496EDF50495C02E1DF6A11D0420E496EB8
:102F7A00DF50495C02E1080E06D0430E496EDF506D
:102F8A00495C03E1100EDF6E02D02C8C28D0010EB2
:102F9A00DB50DF24E96EEA6AD890E936EA36690E30
:102FAA00E926010EEA22020EDBCFEEFF030EDBCF8B
:102FBA00EDFF010EDB50DF24EA6A510FE96E010EC4
:102FCA00EA22EF040AE1010EDB50DF24EA6A510F1C
:102FDA00E96E010EEA22020EEF6EE3EC11F0040E26
:102FEA00E15C02E2E16AE552E16EE552E7CFD9FF20
:102FFA001200E3EF11F0E3EF11F0E3EF11F0E3EF6A
:10300A0011F0E3EF11F0E3EF11F0E3EF11F0E3EF6A
:10301A0011F0E3EF11F0D9CFE6FFE1CFD9FF070EA8
:10302A00E126E66AD9CFE6FFDACFE6FF030EE66EBF
:10303A00E7D9E552E552E552E552E66AD950020F60
:10304A00E66E000EDA20E66E030EE66ED9D9E55278
:10305A00E552E552E5522C5065E1DECF9AF1DDCF1B
:10306A009BF1020EDBCFA2F1030EDBCFA3F1040E1C
:10307A00DB6A030EF36E040EDBCFF4FFF350F45C4D
:10308A004FE2010EE66ED9CFE6FFDACFE6FF030E76
:10309A00E66EB6D9E552E552E552E552E76E050EFF
:1030AA00E7CFDBFF010EE66ED950020FE66E000E87
:1030BA00DA20E66E030EE66EA3D9E552E552E55232
:1030CA00E552E76E060EE7CFDBFF2C502BE1050E2B
:1030DA00DB5026E1060EDB5023E1040EDB28E96E05
:1030EA00EA6AD890E936EA369A0EE926010EEA2209
:1030FA00DECFEEFFDDCFEDFF040EDB28E96EEA6AD4
:10310A00D890E936EA36A20EE926010EEA22020E24
:10311A00DBCFEEFF030EDBCFEDFF040EDB2AA9D7D0
:10312A00E3EC11F0070EE15C02E2E16AE552E16EBE
:10313A00E552E7CFD9FF1200D9CFE6FFE1CFD9FF99
:10314A00E652E66AD9CFE6FFDACFE6FF010EE66E6F
:10315A0057D9E552E552E552E5522C500DE1DF50C0
:10316A0007E0F00E9314936E0101010E996F02D0DD
:10317A000101996BE3EC11F0E552E552E7CFD9FF73
:10318A001200F29EF29C0FEF00F01200D9CFE6FF78
:10319A00E1CFD9FF100EE126E66AD950010FE66E9B
:1031AA00000EDA20E66EE66A2BD9E552E552E552C0
:1031BA00E552E66AD9CFE6FFDACFE6FF010EE66E00
:1031CA001FD9E552E552E552E552E66AD950040F95
:1031DA00E66E000EDA20E66E020EE66E11D9E552B0
:1031EA00E552E552E552E66AD950020FE66E000E44
:1031FA00DA20E66E030EE66E03D9E552E552E55291
:10320A00E552E66AD9500A0FE66E000EDA20E66E3B
:10321A00060EE66EF5D8E552E552E552E552E66A43
:10322A00D950060FE66E000EDA20E66E070EE66E3D
:10323A00E7D8E552E552E552E552E66AD9500E0F53
:10324A00E66E000EDA20E66E040EE66ED9D8E55276
:10325A00E552E552E552E66AD9500F0FE66E000EC6
:10326A00DA20E66E050EE66ECBD8E552E552E55257
:10327A00E552010EDBCF49F04A6A49BE4A6849C0A5
:10328A00E6FF4AC0E6FFAE0E4B6E6C0E4C6E4D6A00
:10329A004BC0E6FFE66E4DC0E6FF31EC38F04E6EED
:1032AA00050EE15E4E50DFCFE6FFE66AA20E496EDA
:1032BA006C0E4A6E4B6A49C0E6FFE66E4BC0E6FFEB
:1032CA0031EC38F04C6E050EE15E4C50040EDBCF4B
:1032DA00E6FF050EDBCFE6FF960E496E6C0E4A6ED0
:1032EA004B6A49C0E6FFE66E4BC0E6FF31EC38F0A8
:1032FA004C6E050EE15E4C50020EDBCFE6FF030E6C
:10330A00DBCFE6FF8A0E496E6C0E4A6E4B6A49C0E5
:10331A00E6FFE66E4BC0E6FF31EC38F04C6E050E68
:10332A00E15E4C50D9500A0FE96EDACFEAFFEECFD0
:10333A00E6FFEECFE6FFEECFE6FFEFCFE6FF7D0E2C
:10334A00496E6C0E4A6E4B6A49C0E6FFE66E4BC088
:10335A00E6FF31EC38F04C6E070EE15E4C50D95066
:10336A00060FE96EDACFEAFFEECFE6FFEECFE6FF11
:10337A00EECFE6FFEFCFE6FF700E496E6C0E4A6E97
:10338A004B6A49C0E6FFE66E4BC0E6FF31EC38F007
:10339A004C6E070EE15E4C500E0EDBCFE6FFE66A7E
:1033AA00640E496E6C0E4A6E4B6A49C0E6FFE66EC1
:1033BA004BC0E6FF31EC38F04C6E050EE15E4C5026
:1033CA000F0EDBCFE6FFE66A580E496E6C0E4A6EA8
:1033DA004B6A49C0E6FFE66E4BC0E6FF31EC38F0B7
:1033EA004C6E050EE15E4C50E3EC11F0100EE15C00
:1033FA0002E2E16AE552E16EE552E7CFD9FF120037
:10340A00D9CFE6FFE1CFD9FF090EE126080EDB6A24
:10341A000D0E496E0401CE51EA6A000FE96E030EE1
:10342A00EA22EF50495C05E1FB0EDB5044E12C88AF
:10343A0042D0CE51EA6A000FE96E030EEA22EF503B
:10344A002C081FE0FB0EDB501AE1CE51EA6A000F8E
:10345A00E96E030EEA22EF50E66EE66A310E496E15
:10346A006C0E4A6E4B6A49C0E6FFE66E4BC0E6FF39
:10347A0031EC38F04C6E050EE15E4C502C8A020E8F
:10348A00E5D1CE2BCE51496E4A6A000E491804E1A5
:10349A00010E4A1801E1CE6B0D0E496ECE51EA6A51
:1034AA00000FE96E030EEA22EF50495C06E1FB0EBB
:1034BA00DB5001E12C88030EC9D12D0E496ECE5185
:1034CA00EA6A000FE96E030EEA22EF50495C2EE128
:1034DA00040E4A6EFE0EDB504A5C28E0050E4B6E67
:1034EA00FE0EDB504B5C22E0FE0EDB0401E147D10D
:1034FA00030E496EFE0EDB50495C01E140D1070E16
:10350A004A6EFE0EDB504A5C01E139D1010EF36EC0
:10351A00080EF3CFDBFFCE2BCE51496E4A6A000E5E
:10352A00491804E1010E4A1801E1CE6B040E496EF6
:10353A00FE0EDB50495C11E0050E4A6EFE0EDB50B2
:10354A004A5C0BE00A0EE66ED9CFE6FFDACFE6FF59
:10355A0089D9E552E552E55242D0CE51EA6A000FC6
:10356A00E96E030EEA22EFCF49F0000E49C0DFFFF1
:10357A00010EDB6A020EDB6A030EDB6A050E496E78
:10358A00FE0EDB50495C1FE1000EDFCFE6FF010EA5
:10359A00DBCFE6FF8AEC39F0E552E552F3CF49F08A
:1035AA00F4CF4AF04B6A4C6A4AAE02D04B684C6878
:1035BA0049C0DFFF010E4AC0DBFF020E4BC0DBFF32
:1035CA00030E4CC0DBFF0401CE2BCE51496E4A6A72
:1035DA00000E491804E1010E4A1801E1CE6B080EEB
:1035EA00DB506FE0FE0EDB500FE1D9CFE9FFDACFF7
:1035FA00EAFFD880800EEE54000EEE54000EEE5410
:10360A00000EEE5401E2BBD0020E496EFE0EDB50F4
:10361A00495C0FE1D9CFE9FFDACFEAFFD880000E83
:10362A00EE54800EEE54000EEE54000EEE5401E2FB
:10363A00A6D0060E4A6EFE0EDB504A5C0FE1D9CFC9
:10364A00E9FFDACFEAFFD880000EEE54000EEE54FE
:10365A00000EEE54800EEE5401E291D0D9CFE9FF6C
:10366A00DACFEAFF040EEECFDBFF050EEECFDBFF6B
:10367A00060EEECFDBFF070EEECFDBFF080EDB50A8
:10368A0001E196D0040EDBCF3BF0050EDBCF3CF018
:10369A00060EDBCF3DF0070EDBCF3EF040684168F7
:1036AA004268436852EC39F0040E37C0DBFF050E5E
:1036BA0038C0DBFF060E39C0DBFF070E3AC0DBFF5E
:1036CA0077D0FE0EDB500EE1D9CFE9FFDACFEAFF61
:1036DA00D8807F0EEE54000EEE54000EEE54000E0B
:1036EA00EE544DE3FE0EDB040EE1D9CFE9FFDACF4B
:1036FA00EAFFD880FF0EEE54000EEE54000EEE5490
:10370A00000EEE543CE3020E496EFE0EDB50495C9D
:10371A000EE1D9CFE9FFDACFEAFFD880FF0EEE54E7
:10372A007F0EEE54000EEE54000EEE5428E3030E04
:10373A004A6EFE0EDB504A5C0EE1D9CFE9FFDACFC2
:10374A00EAFFD880FF0EEE54FF0EEE54000EEE5440
:10375A00000EEE5414E3060E4B6EFE0EDB504B5C6D
:10376A0011E1D9CFE9FFDACFEAFFD880FF0EEE5494
:10377A00FF0EEE54FF0EEE547F0EEE5403E22C8C35
:10378A00010E64D0070E496EFE0EDB50495C10E054
:10379A00D9CFE9FFDACFEAFF040EEECFDBFF050E41
:1037AA00EECFDBFF060EEECFDBFF070EEECFDBFF21
:1037BA00FE0EDB50070A38E0010A25E0050A16E08A
:1037CA00010A14E0030A08E0050A06E0010A04E017
:1037DA00050A02E0040E3AD0FC0EDBCFE9FFFD0E2B
:1037EA00DBCFEAFF040EDBCFEFFF2FD0FC0EDBCFDF
:1037FA00E9FFFD0EDBCFEAFF040EDBCFEEFF050E7D
:10380A00DBCFEDFF22D0FC0EDBCFE9FFFD0EDBCFD5
:10381A00EAFF040EDBCFEEFF050EDBCFEEFF060E4E
:10382A00DBCFEEFF070E0FD0FC0EDBCFE9FFFD0E5C
:10383A00DBCFEAFFDFCFEEFF010EDBCFEEFF020E9A
:10384A00DBCFEEFF030EDBCFEEFF000E496E090E53
:10385A00E15C02E2E16AE552E16E4950E552E7CFE6
:10386A00D9FF1200D9CFE6FFE1CFD9FF020EE12638
:10387A00FD0EDBCFE9FFFE0EDBCFEAFFEE6AEE6A52
:10388A00EE6AEE6A010EDB6AFC0EDB50F36E010E85
:10389A00DBCFF4FFF350F45C62E20401CE51EA6A32
:1038AA00000FE96E030EEA22EFCFDFFF300EDF5C76
:1038BA0051E3DF5039084EE3FD0EDBCFE9FFFE0E80
:1038CA00DBCFEAFFEECF49F0EECF4AF0EECF4BF076
:1038DA00EFCF4CF00A0E406E416A426A436A49C011
:1038EA003BF04AC03CF04BC03DF04CC03EF052ECBD
:1038FA0039F037C049F038C04AF039C04BF03AC005
:10390A004CF0300EDF5C4D6E4E6A4F6A506AE850DA
:10391A0049264E504A224F504B2250504C22FD0EFF
:10392A00DBCFE9FFFE0EDBCFEAFF49C0EEFF4AC05C
:10393A00EEFF4BC0EEFF4CC0EEFF0401CE2BCE5182
:10394A00496E4A6A000E491807E1010E4A1804E155
:10395A00CE6B02D0000E04D0010EDB2A95D7010EE1
:10396A00496E020EE15C02E2E16AE552E16E4950FB
:10397A00E552E7CFD9FF12002550E66EE66A250E1A
:10398A00496E6C0E4A6E4B6A49C0E6FFE66E4BC042
:10399A00E6FF31EC38F04C6E050EE15E4C50120039
:1039AA000501A85108E0010E496E6550020B01E0BD
:1039BA00010E495C1BE10101FA07000EFB5BFC5199
:1039CA000BE1FA51FB1111E18C86A00EFA6F0F0E72
:1039DA00FB6F010EFC6F1200FA51FB1163E18C962A
:1039EA00A00EFA6F0F0EFB6FFC6B1200A80509E020
:1039FA00020EA85D06E0040EA85D03E0100EA85DA5
:103A0A001BE10101FA07000EFB5BFC510BE1FA51C5
:103A1A00FB1111E18C86200EFA6F4E0EFB6F010E20
:103A2A00FC6F1200FA51FB113DE18C96200EFA6FE1
:103A3A004E0EFB6FFC6B1200200EA85D33E10101F4
:103A4A00FA07000EFB5BFC510AE1FA51FB112AE16D
:103A5A008C86100EFA6F270EFB6F010E18D0FC052C
:103A6A000AE1FA51FB111EE18C96100EFA6F270E2D
:103A7A00FB6F020E0CD0020EFC5D0BE1FA51FB113A
:103A8A0011E18C86A00EFA6F860EFB6F030EFC6F97
:103A9A001200FA51FB1106E18C96100EFA6F270EEE
:103AAA00FB6FFC6B1200D9CFE6FFE1CFD9FFE652DC
:103ABA00A098636A626A0F01160E396F9F0E376FFC
:103ACA007B0E366F658C386B030EE66EE66AE66A25
:103ADA00270EE66E0F0EE66EE4EC37F0496E050E21
:103AEA00E15E4950659CDF6ADF50496E4A6A100EF2
:103AFA00495C000E4A5810E2DF50040DF3CFE9FF8B
:103B0A00F4CFEAFF000EE926040EEA22EE6AEE6A14
:103B1A00EE6AEE6ADF2AE8D70F01160E266F62A652
:103B2A0002D06296FCD70501C36BC86BC96BCA6B1E
:103B3A006598DF6A040EDF5C18E2EA6ADF34FE0B7E
:103B4A00EA36E96EB70EE926050EEA22EE6AED6A52
:103B5A00EA6ADF34FE0BEA36E96EAF0EE926050E95
:103B6A00EA22EE6AED6ADF2AE5D70501080EB76F89
:103B7A00040EB86FA96BA86BE552E552E7CFD9FFDF
:103B8A001200D9CFE6FFE1CFD9FFE65282BE06D0B6
:103B9A00656A0F01366B0501A86B8AD00501A85129
:103BAA0010E1656A0F01366B160E396F9F0E376F7B
:103BBA007B0E366F65B602D06586FCD70501010E0D
:103BCA00A86FA8050AE165BA08D0626A0F01366BC8
:103BDA00368136890501020EA86F6250040B06E091
:103BEA000F013651040B02E06294BBD865B260D073
:103BFA006250010B13E00F013651010B0FE053DF46
:103C0A000501040EA86F0401400E026F040E036F33
:103C1A00400E016F006B8C0E001362906250100B05
:103C2A0006E00F013651100B02E088D86298625004
:103C3A00400B14E00F013651400B10E0010EE66E06
:103C4A00E66A000EE66EE66A730EE66EE66A4AEC0D
:103C5A0037F0496E060EE15E4950629C6250200BB5
:103C6A0005E00F013651200B01E04ED86250020BDD
:103C7A0014E00F013651020B10E0010EE66EE66AFF
:103C8A00000EE66EE66AE6687F0EE66E4AEC37F0EC
:103C9A00496E060EE15E4950636A040E0501E76E3D
:103CAA00A819E8AE02D0E73402D0E750A85D02E2D4
:103CBA00A19825D00F0136A721D0DF6A040EDF5C58
:103CCA001DE262A61BD064CFD0F56296780E05017C
:103CDA00D01502E15CD810D0000EE66EE66AD00E6E
:103CEA00E66E050EE66E720EE66EE66A4AEC37F08E
:103CFA00496E060EE15E4950DF2AE0D7A198E552E7
:103D0A00E552E7CFD9FF12000F0126A115D0ABC5A6
:103D1A00E9FFACC5EAFFEF5080080DE1B7C5E9FF3E
:103D2A00B8C5EAFFEF50840806E1ABC5E9FFACC5A8
:103D3A00EAFF8C0EEF6E2691629A12000F01368509
:103D4A0062986582000EE66EE66AE66EE66A750EAF
:103D5A00E66EE66A4AEC37F0496E060EE15E4950B5
:103D6A001200000EE66EE66AE66EE66A740EE66E0B
:103D7A00E66A4AEC37F0496E060EE15E49506592F2
:103D8A000F01369562A402D06294FCD71200D9CFF3
:103D9A00E6FFE1CFD9FFE652FD0E0501D0155AE143
:103DAA007E0ED015E8407F0B040DF3CFABF5F4CFB0
:103DBA00ACF5000EAB27040EAC23ABC5ADF5ACC514
:103DCA00AEF5AD75ABC5E9FFACC5EAFFEF503C0BEC
:103DDA00E842E8420D083CE1ABC5E9FFACC5EAFFA1
:103DEA00020EE926000EEA22EECF49F0EFCF4AF0A2
:103DFA00480E49182BE1040E4A1828E1ABC5E9FF21
:103E0A00ACC5EAFF020EE926000EEA22400EEE6E6B
:103E1A00040EED6EDF6ADF50496E4A6A080E495C8D
:103E2A00000E4A5813E2DF50EA6A480FE96E040EA0
:103E3A00EA22EF50E66EDF50EA6A400FE96E040E9E
:103E4A00EA22E552E750EF6EDF2AE5D70DD807D010
:103E5A002ED805D0FD0ED015040801E14ED8E55242
:103E6A00E552E7CFD9FF1200B7C5E9FFB8C5EAFFA7
:103E7A00EF50800B05E0B7C5E9FFB8C5EAFFEF6A66
:103E8A000501BF6BC06BC46BC56BC36BB5D8000EA5
:103E9A00E66EE66AE66EE66A030EE66EE66A4AECE5
:103EAA0037F0496E060EE15E495096EF21F0020E98
:103EBA000501C05D02E1F1EF22F06CD80501D15194
:103ECA001AE1ADC5E9FFAEC5EAFFEE52400EEF6E4C
:103EDA00ADC5E9FFAEC5EAFF020EE926000EEA22E9
:103EEA00400EEE6E040EED6EADC5E9FFAEC5EAFFFB
:103EFA008C0EEF6E1200D16B1200D9CFE6FFE1CF24
:103F0A00D9FFE652B7C5E9FFB8C5EAFFEF50400B43
:103F1A0001E0010EDF6E0501B775080EA85D0CE120
:103F2A0042C438FF0F013851000803E20501100EA0
:103F3A0002D00501040EA86FC00526E1B7C5E9FF46
:103F4A00B8C5EAFF020EE926000EEA22480EEE6E16
:103F5A00040EED6EB8DA020E0501BF5D06E1B7C5C3
:103F6A00E9FFB8C5EAFF840E0DD0DF5006E1B7C5F8
:103F7A00E9FFB8C5EAFFC80E05D0B7C5E9FFB8C55D
:103F8A00EAFF880EEF6E01D005D8E552E552E7CF79
:103F9A00D9FF1200D9CFE6FFE1CFD9FF020EE12601
:103FAA000501C06BB7C5E9FFB8C5EAFFEF6A040EA1
:103FBA00B719496EB8C54AF0DE6EB8C5DDFFDECF67
:103FCA00E9FFDDCFEAFFEF6AC8AF0CD0CB51CC11C5
:103FDA0007E005D0CCC5FAFF0501CB51F96EFADF2F
:103FEA000501C89F020EE15C02E2E16AE552E16E58
:103FFA00E552E7CFD9FF120004014051600BE842B5
:10400A00E842E842E842E842000901E01200415170
:10401A000C0A50E00B0A3FE00C0A31E0010A22E0E8
:10402A000B0A1EE0020A1CE0030A18E0080A10E064
:10403A00010A0CE00F0A08E0030A01E01200050178
:10404A00C38F080EA86F1200E5EF20F08DEF23F062
:10405A000501A90EC16F050EC26F0CD03CEF21F00D
:10406A0060EF20F044510501C16FC26BAA0EC1274F
:10407A00050EC223C381010EC46FC38F120005014E
:10408A00C38F04014451EA6AAA0FE96E050EEA22B7
:10409A0042C4EFFF1200000EE66EE66AE66EE66ABA
:1040AA00020EE66EE66A4AEC37F0496E060EE15EEB
:1040BA00495012001200D9CFE6FFE1CFD9FF040E12
:1040CA00E1260401420510E140511F0B00090CE1F1
:1040DA000501C38F030E0401415D04E10501010ED0
:1040EA00CF6F02D00501CF6B040142515FE140510D
:1040FA001F0B02085BE144510F0B000957E0050151
:10410A00C38F040144BF0BD044510F0BE96EEA6A16
:10411A00D890E936EA36AF0EE926050E0AD04451A0
:10412A000F0BE96EEA6AD890E936EA36B70EE92645
:10413A00050EEA22EECFDEFFEDCFDDFF030E415D75
:10414A0006E1DECFE9FFDDCFEAFF840E2ED044512F
:10415A000F0B4A6A260F496E0F0E4A22020E49C0F9
:10416A00DBFF030E4AC0DBFF020EDBCFE9FF030EC3
:10417A00DBCFEAFFEF9044AF0CD0DECFE9FFDDCF13
:10418A00EAFFEF6ADF74DECFE9FFDDCFEAFF400E18
:10419A000CD0DECFE9FFDDCFEAFF880EEF6EDF74C9
:1041AA00DECFE9FFDDCFEAFFC80EEF6E040EE15C59
:1041BA0002E2E16AE552E16EE552E7CFD9FF120069
:1041CA00800E0401405D52E10501C00EC36F040177
:1041DA004351030A29E0010A09E0030A45E10501FE
:1041EA00900EC16F710EC26F120E38D04251F66E28
:1041FA00F76AD890F636F736170EF626720EF722B9
:10420A000900F5CFC1F50A00F5CFC2F5020E050186
:10421A00F76AC125F66EC251F7220900F5CFC4F537
:10422A000A00F5CFC5F51200030E425D1AE24251AB
:10423A00F66EF76AD890F636F736190EF626720E2B
:10424A00F7220900F5CFC1F50A00F5CFC2F5C1C5BD
:10425A00F6FFC2C5F7FF0800F5500501C46FC56B2C
:10426A0012000501C36B12000501C36B1200D9CFFE
:10427A00E6FFE1CFD9FF020EE1260401486B496B44
:10428A0040511F0B020A11E0030A0CE0010A35E152
:10429A000501C38F040148810501CF052EE1040100
:1042AA0048832BD00501C38F28D00501C38F040191
:1042BA0044BF0BD044510F0BE96EEA6AD890E93635
:1042CA00EA36AF0EE926050E0AD044510F0BE96E05
:1042DA00EA6AD890E936EA36B70EE926050EEA22E6
:1042EA00EECFDEFFEDCFDDFFDECFE9FFDDCFEAFF68
:1042FA00EF50040B02E0010E486F0501C3AF07D06F
:10430A00480EC16F040EC26FC381020EC46F020E43
:10431A00E15C02E2E16AE552E16EE552E7CFD9FFDC
:10432A00120065980501C3BF47D0C8AF26D0020E58
:10433A00C06FB7C5E9FFB8C5EAFFEE52EF6AB7C565
:10434A00E9FFB8C5EAFFC80EEF6EADC5E9FFAEC515
:10435A00EAFFEE52400EEF6EADC5E9FFAEC5EAFFC9
:10436A00020EE926000EEA22480EEE6E040EED6EEB
:10437A00ADC5E9FFAEC5EAFF7AD0ADC5E9FFAEC566
:10438A00EAFFEE52400EEF6EADC5E9FFAEC5EAFF99
:10439A00020EE926000EEA22400EEE6E040EED6EC3
:1043AA00ADC5E9FFAEC5EAFF8C0EEF6EB7C5E9FFF2
:1043BA00B8C5EAFF840E5CD0C8BF84D0040140AF00
:1043CA0059D00501C4510401465D0501C5510401D6
:1043DA00475904E246C4C4F547C4C5F574D8050173
:1043EA00010EC06FADC5E9FFAEC5EAFFEE52400E41
:1043FA00EF6EADC5E9FFAEC5EAFF020EE926000E73
:10440A00EA22400EEE6E040EED6EADC5E9FFAEC5B2
:10441A00EAFF800EEF6ED16BABC5E9FFACC5EAFFD0
:10442A00EE52400EEF6EABC5E9FFACC5EAFF020ED5
:10443A00E926000EEA22400EEE6E040EED6EABC5C2
:10444A00E9FFACC5EAFF840EEF6E010ED16FB7C566
:10445A00E9FFB8C5EAFF020EE926000EEA22480E75
:10446A00EE6E040EED6EB7C5E9FFB8C5EAFFC80ED9
:10447A00EF6E12000501020EC06FB7C5E9FFB8C59D
:10448A00EAFFEE52EF6AB7C5E9FFB8C5EAFFC80E00
:10449A00EF6EADC5E9FFAEC5EAFFEE52400EEF6E14
:1044AA00ADC5E9FFAEC5EAFF020EE926000EEA2213
:1044BA00480EEE6E040EED6EADC5E9FFAEC5EAFF1D
:1044CA00C80EEF6E1200D9CFE6FFE1CFD9FF020E78
:1044DA00E1260501400EC45D000EC5590DE2C4C5B2
:1044EA00DEFFC5C5DDFFBF5102E1010E03D0BF05E6
:1044FA0006E1020EBF6F03D0400EDE6EDD6AB7C55D
:10450A00E9FFB8C5EAFFEF92B7C5E9FFB8C5EAFF08
:10451A00EF90B7C5E9FFB8C5EAFF010EDB50EF120D
:10452A00B7C5E9FFB8C5EAFFEE52DFCFEFFF000ECD
:10453A00DB50C45F010EDB50C55B480ECD6F040E25
:10454A00CE6FC3B120D0D9CFE9FFDACFEAFFEE5060
:10455A00ED1038E0C1C5F6FFC2C5F7FFC12B000E4A
:10456A00C2230800F550E66ECDC5E9FFCEC5EAFFC5
:10457A00CD2B000ECE23E552E750EF6EDF06010E7B
:10458A00E2E2DB06E0D7D9CFE9FFDACFEAFFEE5065
:10459A00ED1018E0C1C5E9FFC2C5EAFFC12B000E44
:1045AA00C223EF50E66ECDC5E9FFCEC5EAFFCD2B9B
:1045BA00000ECE23E552E750EF6EDF06010EE3E26E
:1045CA00DB06E1D7020EE15C02E2E16AE552E16E46
:1045DA00E552E7CFD9FF1200D9CFE6FFE1CFD9FFE5
:1045EA00020EE126ABC5E9FFACC5EAFFEE52EFCFFA
:1045FA00DFFFDFCF49F049500501C95D000ECA59F6
:10460A0002E2C9C5DFFFDF50496E4A6AE850C95D58
:10461A00C96F4A50CA59CA6F010EDB6ADF50F36E7E
:10462A00010EDBCFF4FFF350F45C16E2010EDB500F
:10463A00EA6A480FE96E040EEA22EF50E66EC6C532
:10464A00E9FFC7C5EAFFC62B000EC723E552E750AC
:10465A00EF6E010EDB2AE2D7000ED880C955000E94
:10466A00CA5527E2ADC5E9FFAEC5EAFFEE52400ED4
:10467A00EF6EADC5E9FFAEC5EAFF020EE926000EF0
:10468A00EA22480EEE6E040EED6EABC5E9FFACC52C
:10469A00EAFFEF50400B06E1ADC5E9FFAEC5EAFF00
:1046AA00C80E05D0ADC5E9FFAEC5EAFF880EEF6EAC
:1046BA0025D0ADC5E9FFAEC5EAFFEE52400EEF6E5A
:1046CA00ADC5E9FFAEC5EAFF020EE926000EEA22F1
:1046DA00400EEE6E040EED6EADC5E9FFAEC5EAFF03
:1046EA00840EEF6ECB51CC1107E005D0CCC5FAFF92
:1046FA000501CB51F96EFADF0501C89F020EE15C94
:10470A0002E2E16AE552E16EE552E7CFD9FF120013
:10471A00D9CFE6FFE1CFD9FFE6520501C38F030ED9
:10472A00E66EE66AE66A270EE66E0F0EE66EE4ECC1
:10473A0037F0496E050EE15E4950DF6ADF50496E77
:10474A004A6A100E495C000E4A5810E2DF50040D06
:10475A00F3CFE9FFF4CFEAFF000EE926040EEA22BE
:10476A00EE6AEE6AEE6AEE6ADF2AE8D7658C010E17
:10477A00E66EE66AE66AAA0EE66E050EE66EE4ECF8
:10478A0037F0496E050EE15E4950659C0501080E39
:10479A00B76F040EB86F000EAB6F040EAC6FABC5EB
:1047AA00ADF5AE6F42C4A9F5A95102E1100E12D0BF
:1047BA00010EE66EE66AA90EE66E050EE66E010EBB
:1047CA00E66EE66A4AEC37F0496E060EE15E49503B
:1047DA000501200EA86FE552E552E7CFD9FF120076
:1047EA00D9CFE6FFE1CFD9FF020EE126000EDE6E39
:1047FA00040EDD6EFD0EDB50E8244B6EFE0EDB5020
:10480A00040DF3504B24040DF350496E4A6A020E0C
:10481A000F0B05E0D8904A324932E806FBE1D890FE
:10482A0049364A36D89049364A36D9CFE9FFDACFDF
:10483A00EAFF4950EE264A50ED22DECFE9FFDDCFEE
:10484A00EAFFEF9EFD0EDB500AE1FE0EEA6ADB3458
:10485A00FE0BEA36E96EAF0EE926050E09D0FE0E0A
:10486A00EA6ADB34FE0BEA36E96EB70EE926050E74
:10487A00EA22DECFEEFFDDCFEDFFDECFE9FFDDCFAF
:10488A00EAFFEF9CDECFE9FFDDCFEAFF040EE9265F
:10489A00000EEA22EF8C020EE15C02E2E16AE552C6
:1048AA00E16EE552E7CFD9FF1200D9CFE6FFE1CF9B
:1048BA00D9FF020EE126FE0EDB504A6A260F496E28
:1048CA000F0E4A2249C0DEFF4AC0DDFFDECFE9FFF4
:1048DA00DDCFEAFFFD0EDBCFEFFFDBA407D0E66AF0
:1048EA00FE0EDBCFE6FF7CDFE552E552FD0EDBA2D2
:1048FA0008D0010EE66EFE0EDBCFE6FF71DFE55251
:10490A00E552020EE15C02E2E16AE552E16EE5522D
:10491A00E7CFD9FF1200D9CFE6FFE1CFD9FF020EC8
:10492A00E126FE0EDB5020E1ADC5E9FFAEC5EAFF88
:10493A00EE52400EEF6EADC5E9FFAEC5EAFF020EBC
:10494A00E926000EEA22400EEE6E040EED6EADC5AB
:10495A00E9FFAEC5EAFF8C0EEF6EB7C5E9FFB8C531
:10496A00EAFF840EEF6E3BD0FD0EDB50E8244B6E5F
:10497A00FE0EDB50040DF3504B24040DF3CF49F027
:10498A00F4CF4AF0000E4926040E4A2249C0DEFF3F
:10499A004AC0DDFF840EDECFE9FFDDCFEAFFE85033
:1049AA00EF12FD0EDB50E8244B6EFE0EDB50040DB9
:1049BA00F3504B24010F040DF3CF49F0F4CF4AF022
:1049CA00000E4926040E4A2249C0DEFF4AC0DDFF16
:1049DA00840EDECFE9FFDDCFEAFFE850EF12020EC8
:1049EA00E15C02E2E16AE552E16EE552E7CFD9FF06
:1049FA001200D9CFE6FFE1CFD9FF020EE126FD0E64
:104A0A00DB500AE0FE0EEA6ADB34FE0BEA36E96E98
:104A1A00B70EE926050E09D0FE0EEA6ADB34FE0B54
:104A2A00EA36E96EAF0EE926050EEA22EECFDEFF80
:104A3A00EDCFDDFFD9CFE9FFDACFEAFFEE50ED1077
:104A4A0003E1F36AF46A44D0DECFE9FFDDCFEAFF7F
:104A5A00020EE926000EEA22FB0EDBCFEEFFFC0E69
:104A6A00DBCFEDFFDECFE9FFDDCFEAFFEE52FA0E34
:104A7A00DBCFEFFF400EDECFE9FFDDCFEAFFE850E4
:104A8A00EF16880EDECFE9FFDDCFEAFFE850EF121E
:104A9A00FD0EDB500AE0FE0EEA6ADB34FE0BEA3654
:104AAA00E96EB70EE926050E09D0FE0EEA6ADB3476
:104ABA00FE0BEA36E96EAF0EE926050EEA22EF741E
:104ACA00DECF49F0DDCF4AF049C0F3FF4AC0F4FF18
:104ADA00020EE15C02E2E16AE552E16EE552E7CFDD
:104AEA00D9FF1200D9CFE6FFE1CFD9FF65A84ED092
:104AFA00FE0EEA6ADB34FE0BEA36E96EB70EE926E9
:104B0A00050EEA22EE50EFCFEAFFE96E400EEE16EE
:104B1A00EE6AEE6AEE6AFE0EEA6ADB34FE0BEA36EB
:104B2A00E96EB70EE926050EEA22EE50EFCFEAFF4C
:104B3A00E96EEE7CFE0EEA6ADB34FE0BEA36E96EBB
:104B4A00B70EE926050EEA22EF74400E496EFE0EF4
:104B5A00EA6ADB34FE0BEA36E96EB70EE926050E81
:104B6A00EA22EE50EFCFEAFFE96E4950EF16FE0E49
:104B7A00EA6ADB34FE0BEA36E96EB70EE926050E61
:104B8A00EA22EE50EFCFEAFFE96EEF7CE552E7CF7B
:104B9A00D9FF1200DACFE4FFE2CFDAFFE9CFE4FF70
:104BAA00EACFE4FFE6529EA071D19E908E0ECE6EA1
:104BBA00CF681850196E1A6A010E1B6E020E1E5C1F
:104BCA000EE104019C519D1104E004019C07000EB2
:104BDA009D5B04019C519D1101E01B6A06D11E04D4
:104BEA0001E097D0105011100AE11250131007E19A
:104BFA001450151004E11650171001E189D0040170
:104C0A00A5510BE018A202D08D8001D08D9018A674
:104C1A0002D08C8E01D08C9E0AD018A202D08C8031
:104C2A0001D08C9018A602D08B8001D08B901050A6
:104C3A0011101DE000500824006E01500920016E79
:104C4A00000ED8800054800E015410E200C000F01B
:104C5A0001C001F0000E005E800E015A010E19100B
:104C6A00196E010E1A6E1006000E115A1B6A1250A6
:104C7A0013101DE002500A24026E03500B20036E2B
:104C8A00000ED8800254800E035410E202C002F0D3
:104C9A0003C003F0000E025E800E035A040E1910C0
:104CAA00196E010E1A6E1206000E135A1B6A1A505A
:104CBA002FE00401A55105E019B0898619B48A804C
:104CCA0004D019B08C8219B48B8400000000000053
:104CDA0000000000000000000000000000000000CA
:104CEA0000000000000000000000000000000000BA
:104CFA0000000000000000000000000000000000AA
:104D0A000401A55103E089968A9002D08C928B9473
:104D1A006CD0030E1E5C33E10401D45105E0A9C432
:104D2A007BF1AAC47CF119D00E01005114E0B3CE74
:104D3A007AFEB4CE7BFEB1CE4AFEB2CE4BFE0E0157
:104D4A00040E326F0E010251031104E1B1CE02FECC
:104D5A00B2CE03FE02D00401A26B899C04019C51CD
:104D6A009D1104E004019C07000E9D5B04019C5107
:104D7A009D1101E01B6A0401010EAB6F36D0040ECF
:104D8A001E5C33E10401D45105E0A7C47BF1A8C439
:104D9A007CF11AD00E01005114E0B5CE7AFEB6CEDF
:104DAA007BFEAFCE4AFEB0CE4BFE0E01040E326F32
:104DBA000E010251031104E1AFCE02FEB0CE03FE92
:104DCA0003D00401010EA26F898C04019C519D112C
:104DDA0004E004019C07000E9D5B04019C519D1197
:104DEA0001E01B6A0401AB6B00D01B504AE01E6A4B
:104DFA001D5047E01C6A040E1C5C3AE21C50E96E26
:104E0A00EA6AD890E936EA36880EE926040EEA22DA
:104E1A00EECF58F0EFCF59F01C50E96EEA6AD890FD
:104E2A00E936EA36080EE926000EEA2258C0EEFFF5
:104E3A0059C0EDFF1C50E96EEA6AD890E936EA36A5
:104E4A00900EE926040EEA22EECF58F0EFCF59F081
:104E5A001C50E96EEA6AD890E936EA36100EE9265D
:104E6A00000EEA2258C0EEFF59C0EDFF1C2AC3D734
:104E7A0098C418F099C41EF09AC49CF49BC49DF47B
:104E8A001D6A80BE03D00401010EB16FE552E5CF61
:104E9A00EAFFE5CFE9FFE5CFDAFF1100010E086E60
:104EAA00096A0A6E0B6A0C6E0D6A0E6E0F6A106A38
:104EBA00116A126A136A146A156A166A176A1D6AEF
:104ECA00CD92CD9ECD9CCD8ACD98CD96CD948E0E89
:104EDA00CE6ECF68CD809F809E909D80806A810E25
:104EEA00926E816A020E936EF19E826A800E946EB1
:104EFA00836A956A846A966A0F01FE0E486F1F0ECE
:104F0A00496F89948C988D8289828C8C8C8A8D8445
:104F1A008B8289968D908A908C9E899C929C0401A2
:104F2A00010EA26FA56F0401D46B0E01006F04017C
:104F3A00AB6FB06BAC6BAD6BAE6BAF6BB16B1200A2
:104F4A00D9CFE6FFE1CFD9FF030EE126DF6A010ED2
:104F5A00DB6A020EDB6AE66AD9CFE6FFDACFE6FF42
:104F6A00010EE66E05EC1AF0E552E552E552E552FD
:104F7A00E66AD950010FE66E000EDA20E66E030EDD
:104F8A00E66E05EC1AF0E552E552E552E5522C5070
:104F9A0001E003D1DF0446E1D950010FE96EDACF0F
:104FAA00EAFFEE50ED1008E10E01006B0401D46B2C
:104FBA0001017B6B7C6BEFD0D950010FE96EDACF20
:104FCA00EAFF010EEE180FE1ED500DE10401010EAA
:104FDA00D46F0E01006B939201015A0501E0DBD0F8
:104FEA00020E5A6FD8D00401D46B9392B3CEE6FF67
:104FFA00B4CEE6FF040EE66EB1CEE6FFB2CEE6FF11
:10500A00010EE66EA1EC35F0496E060EE15E4950DE
:10501A00000EE66EE66A010EE66EFDDAE552E5522C
:10502A00E552B9D0020EDF5C15E1D950010FE96EE5
:10503A00DACFEAFFEE50ED100AE10401010EA56F86
:10504A009590949095929494929A939AA4D00401EC
:10505A00A56BA1D0040EDF5C07E1010EDBCFB1FE28
:10506A00020EDBCFB2FE97D0050EDF5C07E1010E20
:10507A00DBCFAFFE020EDBCFB0FE8DD0060EDF5CBB
:10508A001CE1D950010FE96EDACFEAFF720ED8801F
:10509A00EE542E0EED540AE2720EF36E010EF3CFA9
:1050AA00DBFF2E0EF36E020EF3CFDBFF010EDBCF1A
:1050BA00A9F4020EDBCFAAF46ED0070EDF5C1CE166
:1050CA00D950010FE96EDACFEAFF720ED880EE549A
:1050DA002E0EED540AE2720EF36E010EF3CFDBFFD1
:1050EA002E0EF36E020EF3CFDBFF010EDBCFA7F419
:1050FA00020EDBCFA8F44FD0080EDF5C16E1D950C0
:10510A00010FE96EDACFEAFF180ED880EE54000ECE
:10511A00ED5407E2180EF36E010EF3CFDBFF020E19
:10512A00DB6A010EDBCFABFE36D0090EDF5C16E17F
:10513A00D950010FE96EDACFEAFF060ED880EE5495
:10514A00000EED5407E2060EF36E010EF3CFDBFFFD
:10515A00020EDB6A010EDBCFACFE1DD00A0EDF5C4D
:10516A0007E1010EDBCFB3FE020EDBCFB4FE0DD09A
:10517A000B0EDF5C07E1010EDBCFB3FE020EDBCFC5
:10518A00B4FE09D00C0EDF5C06E1010EDBCFB5FEE2
:10519A00020EDBCFB6FEE3EC11F0030EE15C02E295
:1051AA00E16AE552E16EE552E7CFD9FF1200D9CFA5
:1051BA00E6FFE1CFD9FF0A0EE126020EDB6A030EF3
:1051CA00DB6A040EDB6A050EDB6A060EDB6A070E73
:1051DA00DB6A080EDB6A090EDB6AE66AD9CFE6FFEC
:1051EA00DACFE6FF030EE66E05EC1AF0E552E55259
:1051FA00E552E552E66AD950020FE66E000EDA2051
:10520A00E66E020EE66E05EC1AF0E552E552E5523C
:10521A00E552010EE66ED950040FE66E000EDA2052
:10522A00E66E020EE66E05EC1AF0E552E552E5521C
:10523A00E5522C5023E1080EDBCFE6FF090EDBCF47
:10524A00E6FF060EDBCFE6FF070EDBCFE6FF040E16
:10525A00DBCFE6FF050EDBCFE6FF020EDBCFE6FF74
:10526A00030EDBCFE6FFDECFE6FFDDCFE6FF10D889
:10527A00496E0A0EE15E4950E3EC11F00A0EE15C58
:10528A0002E2E16AE552E16EE552E7CFD9FF120088
:10529A00D9CFE6FFE1CFD9FF1D50FEE1D950FB0F70
:1052AA00E96EFF0EDA20EA6EEE50ED102EE1D950CB
:1052BA00F90FE96EFF0EDA20EA6EEE50ED1025E1E5
:1052CA00D950F70FE96EFF0EDA20EA6EEE50ED10B4
:1052DA001CE1D950F50FE96EFF0EDA20EA6EEE50A6
:1052EA00ED1013E10401020E996F190E3D6E3E6A2C
:1052FA00FD0EDBCF42F0FE0EDBCF43F0AAEC38F016
:10530A003BC09AF43CC09BF4EBD0010E04019A6FA7
:10531A009B6B986B89948C98FB0EDBCF49F0FC0E43
:10532A00DBCF4AF0800E4A1413E0020E9811986FF0
:10533A003D683E68FB0EDBCF42F0FC0EDBCF43F04C
:10534A007DEC38F0FB0E3BC0DBFFFC0E3CC0DBFF04
:10535A00F90EDBCF49F0FA0EDBCF4AF00001800EDE
:10536A004A1414E0080E04019811986F3D683E68CB
:10537A00F90EDBCF42F0FA0EDBCF43F07DEC38F0CA
:10538A00F90E3BC0DBFFFA0E3CC0DBFFFD0EDBCFA4
:10539A004DF0FE0EDBCF4EF04F6A506A190E406E8A
:1053AA00416A426A436A4DC03BF04EC03CF04FC06E
:1053BA003DF050C03EF052EC39F037C04DF038C0E5
:1053CA004EF039C04FF03AC050F0FB0EDBCF49F037
:1053DA00FC0EDBCF4AF04B6A4C6A4AAE02D04B68ED
:1053EA004C680F0ED89049364A364B364C36E8068A
:1053FA00F9E149C03BF04AC03CF04BC03DF04CC01B
:10540A003EF04DC040F04EC041F04FC042F050C097
:10541A0043F0B0EC39F03BC088F43CC089F4010E8B
:10542A0004018827000E8923FB0EDBCF90F4FC0EC3
:10543A00DBCF91F4FD0EDBCF4DF0FE0EDBCF4EF04D
:10544A004F6A506A190E406E416A426A436A4DC0F9
:10545A003BF04EC03CF04FC03DF050C03EF052EC25
:10546A0039F037C04DF038C04EF039C04FF03AC06D
:10547A0050F0F90EDBCF49F0FA0EDBCF4AF04B6A57
:10548A004C6A4AAE02D04B684C680F0ED890493627
:10549A004A364B364C36E806F9E149C03BF04AC079
:1054AA003CF04BC03DF04CC03EF04DC040F04EC009
:1054BA0041F04FC042F050C043F0B0EC39F03BC06D
:1054CA008AF43CC08BF4010E04018A27000E8B2358
:1054DA00F90EDBCF92F4FA0EDBCF93F4010E996F3B
:1054EA00010E1D6EE552E7CFD9FF1200ABC449F099
:1054FA004A6A49BE4A6849C0E6FF4AC0E6FF200E2A
:10550A004B6E6C0E4C6E4D6A4BC0E6FFE66E4DC09C
:10551A00E6FF31EC38F04E6E050EE15E4E50E3EFD9
:10552A0011F0D9CFE6FFE1CFD9FF020EE126F40E42
:10553A00DE6E010EDD6EE66ED9CFE6FFDACFE6FF4C
:10554A00030EE66E05EC1AF0E552E552E552E55215
:10555A002C5015E10401AB0506E1DECFE6FFDDCFF5
:10556A00E6FFE66A06D0DECFE6FFDDCFE6FF010EF4
:10557A00E66E51D8E552E552E552E3EC11F0020E1F
:10558A00E15C02E2E16AE552E16EE552E7CFD9FF5A
:10559A001200D9CFE6FFE1CFD9FF030EE126DF6A79
:1055AA00010EDB6A020EDB6AE66AD9CFE6FFDACFC2
:1055BA00E6FF010EE66E05EC1AF0E552E552E552F9
:1055CA00E552010EE66ED950010FE66E000EDA20A2
:1055DA00E66E030EE66E05EC1AF0E552E552E55268
:1055EA00E5522C500EE1010EDBCFE6FF020EDBCFB7
:1055FA00E6FFDFCFE6FF0FD8E552E552E552E3ECCE
:10560A0011F0030EE15C02E2E16AE552E16EE55255
:10561A00E7CFD9FF1200D9CFE6FFE1CFD9FF1D505E
:10562A00FEE1FE0EDB0403E10401030E02D00401D5
:10563A00040E996F190E3D6E3E6AFC0EDBCF42F0E6
:10564A00FD0EDBCF43F0AAEC38F03BC09AF43CC025
:10565A009BF4010E1D6EE552E7CFD9FF1200D9CF98
:10566A00E6FFE1CFD9FF050EE126E66AD9CFE6FFCC
:10567A00DACFE6FF010EE66E05EC1AF0E552E552C6
:10568A00E552E552E76E040EE7CFDBFFDB5025E17A
:10569A002C5066E10401A5511AE0DF50000815E21A
:1056AA008994DF0402E18D828982020EDF5C02E1C5
:1056BA008D928982030EDF5C02E18D828992040E4B
:1056CA00DF5C0BE18D92899208D0898406D0DF5085
:1056DA00000802E2899A01D0898A010EE66ED95041
:1056EA00010FE66E000EDA20E66E010EE66E05EC9C
:1056FA001AF0E552E552E552E552E76E040EE7CF9D
:10570A00DBFFDB502BE12C502BE10401A5511FE0FC
:10571A00010EDB50000819E28C98010EDB0402E14D
:10572A008C8C8C8A010EDB50020802E18C9C8C8ADC
:10573A00010EDB50030802E18C8C8C9A010EDB50BF
:10574A0004080CE18C9C8C9A09D08C8807D0010E35
:10575A00DB50000802E28A9A01D08A8AE3EC11F04F
:10576A00050EE15C02E2E16AE552E16EE552E7CF3D
:10577A00D9FF1200FE0E0401AC5DFF0EAD59FF0EFB
:10578A00AE59FF0EAF5905E2AC2B000EAD23AE2386
:10579A00AF23E3EF11F00401AC51AD11AE11AF111B
:1057AA0005E0AC07000EAD5BAE5BAF5BE3EF11F05B
:1057BA00D9CFE6FFE1CFD9FF050EE126E66AD9CFB8
:1057CA00E6FFDACFE6FF070EE66E05EC1AF0E552C1
:1057DA00E552E552E552E76E040EE7CFDBFFDB50F8
:1057EA000BE1DFCFACF4010EDBCFADF4020EDBCF61
:1057FA00AEF4030EDBCFAFF4E3EC11F0050EE15C7F
:10580A0002E2E16AE552E16EE552E7CFD9FF120002
:10581A00ACC4E6FFADC4E6FFAEC4E6FFAFC4E6FF24
:10582A00170E496E6C0E4A6E4B6A49C0E6FFE66E69
:10583A004BC0E6FF31EC38F04C6E070EE15E4C507F
:10584A00E3EF11F0E66AB00EE66E040EE66E010EA4
:10585A00E66E05EC1AF0E552E552E552E5522C5097
:10586A0001E01200E3EF11F0B0C449F04A6A49BE00
:10587A004A6849C0E6FF4AC0E6FF100E4B6E6C0E3E
:10588A004C6E4D6A4BC0E6FFE66E4DC0E6FF31EC4A
:10589A0038F04E6E050EE15E4E50E3EF11F0B1C4E2
:1058AA0049F04A6A49BE4A6849C0E6FF4AC0E6FF6B
:1058BA000A0E4B6E6C0E4C6E4D6A4BC0E6FFE66EDE
:1058CA004DC0E6FF31EC38F04E6E050EE15E4E50EB
:1058DA000401B16BE3EF11F0ADEC31F0FB0EDBCF5D
:1058EA00F3FFDB06F35000090AE0FBEC31F0FA0E95
:1058FA0066EC32F0F3E14A1CF1E1010E01D0000E30
:10590A00DCEF31F0ADEC31F03B0EE12402E3E1686B
:10591A00E652E16E010EDB6A020EDB6AF90EDBCF9C
:10592A00F6FFFA0EDBCFF7FFFB0EDBCFF8FF08001E
:10593A00F550DF6EDF5002E100EF31F0250EDF5C3B
:10594A0002E0F3EF30F0030EDB6A040EDB6A050EA9
:10595A00DB6A060EDB6A070EDB6A15EC31F02D0EE8
:10596A00DF5C0CE02B0EDF5C09E0200EDF5C06E05A
:10597A00230EDF5C03E0300EDF5C1AE1DF50300AF1
:10598A0014E0130A0FE0030A0AE00B0A05E0060A0C
:10599A00E4E1030EDB80E1D7030EDB82DED7030EE0
:1059AA00DB84DBD7030EDB86D8D7030EDB88D5D79B
:1059BA002A0EDF5C1BE111EC31F05FEC31F010E0F4
:1059CA00030EDB803D683E68130EDBCF42F0140EF7
:1059DA00DBCF43F07DEC38F0040E3BC0DBFF03D095
:1059EA00130E48EC31F015EC31F00BD0090EDB6ADE
:1059FA00B6EC31F003E02AEC32F0FAD7090E48ECA3
:105A0A0031F0030EDBB0DB982E0EDF5C1BE115ECE8
:105A1A0031F02A0EDF5C0BE111EC31F05FEC31F072
:105A2A0003E1130E9AEC31F015EC31F00BD0090EAC
:105A3A00DB6AB6EC31F003E02AEC32F0FAD7090E51
:105A4A009AEC31F0680EDF5C07E115EC31F0680E74
:105A5A00DF5C1DE1030E18D0740EDF5C17E07A0ECE
:105A6A00DF5C14E0480EDF5C06E0540EDF5C03E006
:105A7A005A0EDF5C02E1020E07D06C0EDF5C03E017
:105A8A006A0EDF5C04E1010EEDEC31F0C9DBDF5098
:105A9A006E0A01E17FD31E0A01E192D1200A01E1D7
:105AAA008FD13F0A01E149D11A0A01E146D10D0A13
:105ABA0001E143D1200A01E140D13A0A01E13DD195
:105ACA00200A01E13AD1260A01E135D10D0A01E1A4
:105ADA0032D11A0A01E1D9D0200A4AE0300A1FE07D
:105AEA00460A0EE0250A01E083D3D950F90FE96E80
:105AFA00FF0EDA20EA6E010EEE5E000EEE5AEE5A44
:105B0A00FBEC31F0250EE66E95DB03E14A1C01E160
:105B1A0069D3F7EC31F001E26BD3DB2A69D3080EC3
:105B2A00DB6A040EDB50010806E2040EDB04BFEC5C
:105B3A0031F0DB508BDB080EDB5009E0030EDB5043
:105B4A00010B05E172DB01E04DD3080EDB6A64DB71
:105B5A00EFCFDFFF6FEC32F003E14A1C01E142D3E1
:105B6A00F7EC31F001E3DB2A60DB01E141D33AD300
:105B7A00070EDB5002080FE13BEC32F0030E02EC99
:105B8A0032F00E0EEECFDBFF0F0EEECFDBFF100E64
:105B9A00EECFDBFF20D0F70EDBCF4CF0F80EDBCFD9
:105BAA004DF0020E4C5E000E4D5AF70E4CC0DBFF54
:105BBA00F80E4DC0DBFF4CC0E9FF4DC0EAFFF2EC26
:105BCA0031F04B6A0E0E49C0DBFF0F0E4AC0DBFFF5
:105BDA00100E4BC0DBFF0E0EDBCFE6FF0F0EDBCF46
:105BEA00E6FF100EDBCFE6FF0CEC38F0E552E5528B
:105BFA00E552130E3CC0DBFF140E3DC0DBFF060E60
:105C0A00DB5005E0130E36EC32F001E26ADB5AECA7
:105C1A0032F002E2130E37DB1DEC32F006E0040E1E
:105C2A0036EC32F002E2050E2EDB030EDBB005D0B5
:105C3A00FCDA01E0D7D2080EDB6A090EDB6A0E0E27
:105C4A00DBCFF6FF0F0EDBCFF7FF100EDBCFF8FF2F
:105C5A000800F550DF6EDF5014E060EC32F011E21C
:105C6A006FEC32F003E14A1C01E1BCD2BBDB01E379
:105C7A00DB2A090EDB2AD9500E0FE96E000ECBDBA8
:105C8A00E7D7D3DA01E1B4D2ADD2C6DA110EEECF3C
:105C9A00DBFF120EEDCFDBFF110EDBCFE6FF120E9C
:105CAA00DBCFE6FFFEEC37F0E552E552130EF3CFF9
:105CBA00DBFF140EF4CFDBFF060EDB5004E0130EFD
:105CCA00D0DB01E20EDB5AEC32F002E2130EDBDA31
:105CDA00AFDB05E0040EC5DB02E2050ED4DA030EE3
:105CEA00DBB005D0A2DA01E07DD2080EDB6A090E2C
:105CFA00DB6A110EDBCFE9FF120EDBCFEAFFEFCF33
:105D0A00DFFFDF5014E0D7DB12E2E4DB03E14A1CD9
:105D1A0001E168D267DB01E3DB2A090EDB2A110EF7
:105D2A00DB2ADBCFE9FF120EE8E3DB2AE6D77DDACE
:105D3A0001E15ED257D2030EDB8E070EDB0410E1BF
:105D4A0095DB040E5ADB0A0EEECFDBFF0B0EEECF0D
:105D5A00DBFF0C0EEECFDBFF0D0EEECFDBFF6CD0C0
:105D6A00070EDB5003082CE1030EDBAE0DD0B2DACE
:105D7A00020E76DAEFCF49F04A6A4B6A4C6A49AEAC
:105D8A0039D04A684B6835D0F70EDBCF4AF0F80EA7
:105D9A00DBCF4BF0020E4A5E000E4B5AF70E4AC09A
:105DAA00DBFFF80E4BC0DBFF4AC0E9FF4BC0EAFF3E
:105DBA00EFCF49F00A0E49C0DBFF0B0EDB6A38D081
:105DCA00070EDB50020809E1030EDBAE04D059DBF3
:105DDA004BAE10D00ED055DB0DD0030EDBAE12D079
:105DEA0079DA020E3DDAF9DA4B6A4C6A4AAE02D027
:105DFA004B684C68E2DA0C0E4BC0DBFF0D0E4CC050
:105E0A00DBFF1AD0F70EDBCF4BF0F80EDBCF4CF0EE
:105E1A00020E4B5E000E4C5AF70E4BC0DBFFF80E1B
:105E2A004CC0DBFF4BC0E9FF4CC0EAFFD6DAC5DA4B
:105E3A000C0EDB6A0D0EDB6A060EDB5005E1010E65
:105E4A00F36E050EF3CFDBFF150EDB6A160EDB6A67
:105E5A00D950370F496E000EDA204A6E390E49C002
:105E6A00DBFF3A0E4AC0DBFF380EDB6A080EDB6A3C
:105E7A000A0EAEDADF50780A12E0200A10E0280A89
:105E8A000CE0200A0AE03F0A06E00D0A02E0200AB6
:105E9A0008E1020E05D0080E03D0080EDF26100E08
:105EAA0097DA030EDBBE02D0DB92DB94DB50800B69
:105EBA0024E08ADAD890030EEB50000A08E6000EB6
:105ECA00EE5C000EEE58000EEE58000EEE5815E28B
:105EDA0013DA406841684268436852EC39F00A0EA6
:105EEA0037C0DBFF0B0E38C0DBFF0C0E39C0DBFFFF
:105EFA000D0E3AC0DBFF2D0E08D0030EDBA202D036
:105F0A002B0E03D0DBA408D0200EF36E170EF3CFAE
:105F1A00DBFF150EDB2A02D0170EDB6A050EDB50FB
:105F2A0003E1B7D901E189D02C0E496E740E4A6E8D
:105F3A00000E4B6E070EDBCF4CF04D6A4E6A4F6A6D
:105F4A004CC040F04DC041F04EC042F04FC043F04B
:105F5A00D3D9B0EC39F049503724F36E4A5038207F
:105F6A00F46E4B503920F86EF4CFF7FFF3CFF6FFFB
:105F7A000800090EF5CFDBFF580EDF5C0FE1610E5A
:105F8A00F36E090E7BD90AE3200E496E090EDBCFA8
:105F9A00E7FF4950E75E090EE7CFDBFF070EDBCFCD
:105FAA0049F04A6A4B6A4C6A0FDA49C040F04AC063
:105FBA0041F04BC042F04CC043F0EECF3BF0EECF85
:105FCA003CF0EECF3DF0EFCF3EF0B0EC39F03EC002
:105FDA00EDFF3DC0EDFF3CC0EDFF3BC0EFFF390ECA
:105FEA00DBCFE9FFDB063A0EDBCFEAFF01E2DB0695
:105FFA00090EDBCFEFFF150EDB2A4BD995E1030E15
:10600A00DBA61DD06F0EDF5C06E1C1D918E3150EC1
:10601A00DB285BDA14D0780EDF5C09E0580EDF5C0F
:10602A0006E0620EDF5C03E0420EDF5C08E1020E6E
:10603A00F36E160EF3CFDBFF02D0150EDB6A030EEA
:10604A00DB50100B0EE0040EDBCF49F0050EDB50DF
:10605A00D880495406E2060EDB5003E1040EDB50F9
:10606A0034DA95D90AE2050EDBCFE7FF150EDB50CD
:10607A00E75E050EE7CFDBFF02D0050EDB6A040EF2
:10608A00DBCF49F0160E45D9D880495414E2160ED2
:10609A00DBCFE6FF150EDBCFE6FF040EDBCFE6FF14
:1060AA00050EDB50E552E75CE552D880E754E5522D
:1060BA00D880E7545FD9030EDB50010B0BE1080EC1
:1060CA00DB5008E0B2D801E08DD0080EDB50BED814
:1060DA00080EDB6A170EDB5007E088D9170EF1D9D4
:1060EA0003E14A1C01E17ED0160EDB5016E07ED990
:1060FA00300EE66E9FD802E14A1C74E077D9DFCFF2
:10610A00E6FF10EC39F0E552E552E552F4CF4AF0D9
:10611A000001F31C02E14A1C65E0050EDBCF49F0E1
:10612A00160EDB50D880495409E2050EDBCFE7FF93
:10613A00160EDB50E75E050EE7CFDBFF300EE66E8C
:10614A00050ECBD94FE1390EDB2ADBCFE9FF3A0E38
:10615A0001E3DB2ADBCFEAFF090EEFCFDBFFDB50DF
:10616A000EE044D9090EADD902E14A1C3BE0390ED2
:10617A00DB2ADBCFE9FF3A0EEDE3DB2AEBD755D872
:10618A0031E1160EDBCFE6FF080EC3D8E552E7244D
:10619A005DD82ED0070EDB50030A1CE0010A14E07A
:1061AA00030A07E07BD9DBCFEEFF020EDBCFEDFF60
:1061BA001FD0F5D84E6A4CAE02D04D684E682CD826
:1061CA00BCD84EC0EEFF14D0EAD84CBE4D6824D8D5
:1061DA00B4D80ED063D9DBCFEFFF0AD07BD905E163
:1061EA004A1C03E1F368F46810D0FCD801E3DB2A07
:1061FA0079D99CEF2CF0010EDBCF49F0020EDBCFF0
:10620A004AF049C0F3FF4AC0F4FF3B0EE15C02E2E8
:10621A00E16AE552E16ECBD029D9020E02EF32F0E3
:10622A0061D90800F550DF6E1200200EE66E080EE6
:10623A0072EF32F010EC39F0E552E552E552F3CF45
:10624A0049F0F4CF4AF00001F31C1200496E4A6A81
:10625A00D950010F4DD94950EE264A50ED2212006D
:10626A004D5E000E4E5AF70E4DC0DBFFF80E4EC0C3
:10627A00DBFF4DC0E9FF4EC0EAFF1200DBCFF4FF9F
:10628A00F350F45C1200DB50E76E040EE7CFDBFF3D
:10629A0012000A0EDBCF49F00B0EDBCF4AF00C0ED0
:1062AA00DBCF4BF00D0EDBCF4CF049504A104B10B0
:1062BA004C101200130EEECFDBFF140EEDCFDBFFF6
:1062CA00130EDBCF49F0140EDBCF4AF00001800E2B
:1062DA004A141200F70EDBCF4DF0F80EDBCF4EF06A
:1062EA001200050EDB50E66ED950130F01D9E552A4
:1062FA00E750EE6EED6A12000A0EDBCF3BF00B0E92
:10630A00DBCF3CF00C0EDBCF3DF00D0EDBCF3EF0C9
:10631A001200DBCFE6FF150EDBCFE6FF050EDB50E2
:10632A00E552E724E552E7241200DB50CED8010EED
:10633A00F36E060EF3CFDBFF1200EE50EFCFEAFF4B
:10634A00E96E4BC0EEFF4CC0EEFF4DC0EEFF1200EF
:10635A00D9CFE6FFDACFE6FFE1CFD9FFE2CFDAFF06
:10636A001200DFCFE6FFE66A9EEC39F0E552E5520D
:10637A00F3501200E76E080EE7CFDBFF1200EECFF4
:10638A0049F0EECF4AF0EFCF4BF04C6A1200050EFF
:10639A00DBCF49F0150EDB50D88049541200010EAC
:1063AA00DBCF4BF0020EDBCF4CF04D6A1200E55208
:1063BA00E5CFDAFFE7CFD9FF12000A0E49C0DBFFAB
:1063CA000B0E4AC0DBFF1200D9500A0F7DEF32F0E4
:1063DA00F36E070EF3CFDBFF1200EECF49F0EFCFDB
:1063EA004AF01200010EDB2A020E1200FC0EDBCF6D
:1063FA00E6FFFD0EDBCFE6FF1200495E000E4A5AA9
:10640A00F70E49C0DBFFF80E4AC0DBFF49C0E9FFBF
:10641A004AC0EAFF1200DA20EA6EEF2AEECFF6FF50
:10642A00000EEF22EECFF7FFEF22EECFF8FF1200B9
:10643A00040EDBCFE6FF130EDB50E552E75C9ADF72
:10644A00DB5004DF060EDB501200090EDB500A0D8A
:10645A00F350DF24D00FE76E090EE7CFDBFF15EF0D
:10646A0031F0DB50F36E050E43EF31F0F70EDBCF60
:10647A0049F0F80EDBCF4AF01200DFCFE6FF1FEF3C
:10648A0031F028DF030EECDEC4EF31F071EC2CF0B2
:10649A00E552E552E552E55200091200BDDEEE5022
:1064AA00EFCFEAFFE96E010E1200130EDB50F36E16
:1064BA00040E43EF31F0040EDB50F36E090E43EF86
:1064CA0031F0DBCFE6FF1FEF31F0E76E050EE7CFC5
:1064DA00DBFF12008BDF42EF32F0DBCFE6FF86DF15
:1064EA004BEF32F0D950F90FE96EFF0E10EF32F090
:1064FA00E96E000EDA20EA6E1200040140511F0B09
:10650A00010801E012004051600BE842E842E8420B
:10651A00E842E842010801E01200445103E0440560
:10652A0001E012004151220A31E0030A24E0010A83
:10653A0015E0210A0DE0010A01E012000501A00E92
:10654A00C16F050EC26F080EC46FC56BC38121D01F
:10655A000501A00EC16F050EC26F1BD046C4C9F556
:10656A0047C4CAF50501880EC66F050EC76FCB6B07
:10657A00CC6BC88F12000501880EC16F050EC26F61
:10658A00070EC46FC56BC10EC36F120042C49BF5E0
:10659A000501C38F12000501886B4B0E896F8A6B48
:1065AA008B6B8C6B8D6B080E8E6F906B8F6B1A0ECC
:1065BA00E66E020EE66E5AEC24F0E552E5521E0E25
:1065CA00E66E030EE66E5AEC24F0E552E552400EF2
:1065DA00E66E080EE66E050EE66EE66A030EE66ED7
:1065EA00FEEC24F0496E050EE15E4950F3CF97F5B3
:1065FA00F4CF98F50501996B9A6B1200D9CFE6FF93
:10660A00E1CFD9FF05018F6B9751981102E1000E76
:10661A0008D097C5E9FF98C5EAFFEF50800B01E063
:10662A00010E000945E1FC0EDBCF49F097C5E9FFF1
:10663A0098C5EAFFEE52EF50D880495408E297C550
:10664A00E9FF98C5EAFFEE52FC0EEFCFDBFF8F6B36
:10665A00FC0EDB508F5D19E28F51EA6A080FE96E72
:10666A00050EEA22EF50E66E8F51E76EFD0EDBCF84
:10667A00E9FFFE0EDBCFEAFFE750E926000EEA2229
:10668A00E552E750EF6E8F2BE3D7400EE66E080E09
:10669A00E66E050EE66EE66A030EE66EFEEC24F082
:1066AA00496E050EE15E4950F3CF97F5F4CF98F5A0
:1066BA0005018F51E552E7CFD9FF1200D9CFE6FF86
:1066CA00E1CFD9FF050190510CE1FD0EDBCF91F529
:1066DA00FE0EDBCF92F5FC0EDBCF95F5010E966F21
:1066EA00906FE552E7CFD9FF1200D9CFE6FFE1CF8D
:1066FA00D9FF030EE126050190512DE1DF6AFD0E57
:10670A00DBCF3DF0FE0EDBCF3EF0DE523DC0DEFFBA
:10671A003EC0DDFFDD52DF2ADF50496E4A6AFF0EB6
:10672A00491802E14A500BE0010EDBCFE9FFDB2AF0
:10673A00020EDBCFEAFF01E3DB2AEF50ECE1FD0EAC
:10674A00DBCF91F5FE0EDBCF92F5DFCF95F5050194
:10675A00010E966F906F030EE15C02E2E16AE55268
:10676A00E16EE552E7CFD9FF1200D9CFE6FFE1CFBC
:10677A00D9FF030EE126050190512EE1DF6AFD0ED5
:10678A00DBCF3DF0FE0EDBCF3EF0DE523DC0DEFF3A
:10679A003EC0DDFFDD52DF2ADF50496E4A6AFF0E36
:1067AA00491802E14A500CE0010EDBCFF6FFDB2A62
:1067BA00020EDBCFF7FF01E3DB2A0800F550EBE11D
:1067CA00FD0EDBCF91F5FE0EDBCF92F5DFCF95F50F
:1067DA000501966B010E906F030EE15C02E2E16A1D
:1067EA00E552E16EE552E7CFD9FF1200D9CFE6FFB5
:1067FA00E1CFD9FF020EE126050199519A1102E172
:10680A00000E08D099C5E9FF9AC5EAFFEF50800B40
:10681A0001E0010E000901E084D0030E905D01E160
:10682A00906B905101E17DD0020E905D16E1E66A0F
:10683A00000EE66EE66A010EE66E030EE66EFEECEA
:10684A0024F0496E050EE15E4950F3CF99F5F4CF75
:10685A009AF50501030E906F64D0900562E1400E2F
:10686A00496E4A6A9551495C000E4A5803E2400E45
:10687A00DF6E02D095C5DFFFDF50955D956F480E3C
:10688A00936F050E946F010EDFCFDBFF965116E171
:10689A00010EDB5028E091C5F6FF92C5F7FF08000C
:1068AA00F55093C5E9FF94C5EAFFEF6E932B000EEE
:1068BA009423912B9223010EDB06EAD7010EDB50BB
:1068CA0012E091C5E9FF92C5EAFFEF5093C5E9FFCF
:1068DA0094C5EAFFEF6E932B000E9423912B92231B
:1068EA00010EDB06EBD70501955107E1400EDF5C8F
:1068FA0002E1020E01D0030E906FDFCFE6FF480ED1
:10690A00E66E050EE66E010EE66E030EE66EFEEC10
:10691A0024F0496E050EE15E4950F3CF99F5F4CFA4
:10692A009AF5020EE15C02E2E16AE552E16EE55295
:10693A00E7CFD9FF1200D9CFE6FFE1CFD9FFE65260
:10694A000E01006B016BAA6BDF6A180EDF5C2AE28C
:10695A00EA6ADF34FE0BEA36E96E020EE9260E0E0B
:10696A00EA22EE6AED6ADF50EA6A320FE96E0E0E2B
:10697A00EA22EF6AEA6ADF34FE0BEA36E96E4A0E69
:10698A00E9260E0EEA22EE6AED6AEA6ADF34FE0BA7
:10699A00EA36E96E7A0EE9260E0EEA22EE6AED6A08
:1069AA00DF2AD3D70E01C60EAD6F0E0EAE6F3F0EA5
:1069BA0079140009796ECF0E79140009796E7982FB
:1069CA007B6A7A6A79900F0152815293F00EB4145D
:1069DA000909B46E0E01070EAB6F030EAC6FE00E21
:1069EA00B16F2E0EB26F800EAF6F3E0EB06F040104
:1069FA00D46B93920E01010E006F900EB36F010ECD
:106A0A00B46F900EB56F010EB66FB3CEE6FFB4CE7B
:106A1A00E6FF040EE66EB1CEE6FFB2CEE6FF010E49
:106A2A00E66E8AD8496E060EE15E4950000EE66EA1
:106A3A00E66A010EE66E10EC2BF0E552E552E552DD
:106A4A00E552E552E7CFD9FF1200D9CFE6FFE1CFF1
:106A5A00D9FF050EE126DF6A010EDB6A020EDB6A48
:106A6A00030EDB6A040EDB6AE66AD9CFE6FFDACFE9
:106A7A00E6FF010EE66E05EC1AF0E552E552E55224
:106A8A00E552010EE66ED950010FE66E000EDA20CD
:106A9A00E66E030EE66E05EC1AF0E552E552E55293
:106AAA00E552010EE66ED950030FE66E000EDA20AB
:106ABA00E66E010EE66E05EC1AF0E552E552E55275
:106ACA00E552010EE66ED950040FE66E000EDA208A
:106ADA00E66E030EE66E05EC1AF0E552E552E55253
:106AEA00E5522C501FE1DF50180804E3030EDB5077
:106AFA00180802E22C8C16D0040EDBCFE6FFE66AF9
:106B0A00030EDBCFE6FF010EDBCFE6FF020EDBCF83
:106B1A00E6FFDFCFE6FF10D8496E060EE15E495068
:106B2A00E3EC11F0050EE15C02E2E16AE552E16E86
:106B3A00E552E7CFD9FF1200D9CFE6FFE1CFD9FF5F
:106B4A00FE0EDB5003E10E01006B56D0FE0EDB5049
:106B5A00180852E3FB0EDB5018084EE30E01010E33
:106B6A00006FFE0EDB04E96EEA6AD890E936EA366F
:106B7A007A0EE9260E0EEA22F90EDBCFEEFFFA0EA6
:106B8A00DBCFEDFFFE0EDB04E96EEA6AD890E93648
:106B9A00EA364A0EE9260E0EEA22FC0EDBCFEEFF9B
:106BAA00FD0EDBCFEDFFFE0EDB04EA6A320FE96E63
:106BBA000E0EEA22FB0EDBCFEFFFFE0EDB04E96EC0
:106BCA00EA6AD890E936EA36020EE9260E0EEA2279
:106BDA00EE50ED1011E1FE0EDB04E96EEA6AD89080
:106BEA00E936EA36020EE9260E0EEA22FC0EDBCF61
:106BFA00EEFFFD0EDBCFEDFFE552E7CFD9FF120026
:106C0A002531690D0A00253033690D0A0025303116
:106C1A00306C750D0A0025640A0D00537461747591
:106C2A00733D25690D0A002135204572723A204EBE
:106C3A0065656420636F6D6D61206E6578742C20C4
:106C4A00666F756E643A20272563270D0A00506126
:106C5A0072616D383D25630D0A00506172616D37AE
:106C6A003D25630D0A00506172616D363D256C75D4
:106C7A000D0A00506172616D353D256C640D0A0084
:106C8A00506172616D343D25750D0A005061726163
:106C9A006D333D25640D0A00506172616D323D25E8
:106CAA00640D0A00506172616D313D25640D0A0060
:106CBA0050492C2531750D0A004D522C253033755B
:106CCA000D0A002C25303475004100492C2530333B
:106CDA00692C253033692C253033692C25303369EA
:106CEA002C253033690D0A002138204572723A206A
:106CFA00556E6B6E6F776E20636F6D6D616E64207B
:106D0A0027256325633A253258253258270D0A006C
:106D1A002138204572723A20556E6B6E6F776E205D
:106D2A00636F6D6D616E64202725633A253258279B
:106D3A000D0A002137204572723A20457874726133
:106D4A00207061726D617465720D0A0021362045EA
:106D5A0072723A20496E76616C6964207061726160
:106D6A006D7465722076616C75650D0A0021342098
:106D7A004572723A204D697373696E672070617249
:106D8A00616D657465722873290D0A0021332045E7
:106D9A0072723A20525820427566666572206F7682
:106DAA00657272756E0D0A002132204572723A20A0
:106DBA00545820427566666572206F7665727275E0
:106DCA006E0D0A002131204572723A2043616E2706
:106DDA0074207374657020746861742066617374BA
:106DEA000D0A002130200D0A002008002573001B1F
:0B6DFA005B421B5B314B1B5B30470012
:106E060005D8C6EC1DF007EC0DF0FBD7D9CFE6FF91
:106E1600E1CFD9FF020EE1260F0148694969600EEC
:106E2600D36E9B8C580EDE6E020EDD6EDFCF49F000
:106E3600DF06010EDBCF4AF001E2DB0649504A10BD
:106E4600F5E1948E46EC0CF058EC1DF0020EE15C78
:106E560002E2E16AE552E16EE552E7CFD9FF1200A0
:106E6600120012001200120082EF32F01200D0EF70
:106E760032F065840101080EFD6F070EFE6FFD07F7
:106E8600000EFE5BFD51FE11FAE165941200D9CFAA
:106E9600E6FFE1CFD9FFFD0EDBCF3DF0FE0EDBCFE7
:106EA6003EF0720E3D1801E13E5033E0E8683D18B1
:106EB60002E17F0E3E182BE0740E3D1801E13E50B4
:106EC60024E0750E3D1801E13E501DE0730E3D189D
:106ED60001E13E5016E0030E3D1801E13E500FE081
:106EE600020E3D1801E13E5008E0010E3D1801E199
:106EF6003E5001E010D0BBDF0FD0B8DF0DD0B4DFBD
:106F06000BD0B0DF09D0ACDF07D0ABDF05D0ABDFED
:106F160003D0000001D000D0010E00D0E552E7CF2B
:106F2600D9FF12002A0EF66E100EF76E000EF86EDE
:106F360005010900F550E36F0900F550E46F03E120
:106F4600E36701D03DD00900F550DE6F0900F5502A
:106F5600DF6F0900F550E06F09000900F550E96E92
:106F66000900F550EA6E090009000900F550E16FC5
:106F76000900F550E26F09000900F6CFE5F5F7CFF5
:106F8600E6F5F8CFE7F5DEC5F6FFDFC5F7FFE0C5A6
:106F9600F8FF0501E15302E1E25307E00900F5506D
:106FA600EE6EE107F8E2E207F9D7E5C5F6FFE6C5BA
:106FB600F7FFE7C5F8FF0501E307000EE45BBFD75F
:106FC6001200FE0EE3CFE9FFFF0EE3CFEAFFE9CFA3
:106FD600F3FFEACFF4FFFB0EE35003E1FC0EE350B0
:106FE60009E0FB0EE30602E2FC0EE306FD0EE350AB
:106FF600EE6EF1D71200FE0EE3CFE9FFFF0EE3CFF0
:10700600EAFFF36AF46AEE5203E0F34AF42AFBD786
:107016001200FF0EE3CFF8FFE552FF0EE3CFF7FFB6
:10702600E552FF0EE3CFF6FFE552E66AE66AE66A48
:107036000900F55209E0FD0EE32A05E1FE0EE32AFA
:1070460002E1FF0EE32AF4D7FD0EE3CF3CF0FE0E7D
:10705600E3CF3DF0FF0EE3CF3EF01200D9CFE6FFBF
:10706600DACFE6FFE1CFD9FFE2CFDAFFE652E6520A
:10707600E652E652D950FB0F496EFF0EDA204A6EF1
:1070860049C0DEFFDD6EDECFE6FFDDCFE6FFFB0E9D
:10709600DBCFE6FFFC0EDBCFE6FFFD0EDBCFE6FF28
:1070A600B7CEE6FFB8CEE6FF87EC2CF0496E070EAA
:1070B600E15C02E2E16AE552E16E4950020EF3CF6D
:1070C600DBFF030EF4CFDBFF020EDBCF49F0030E2E
:1070D600DBCF4AF049C0F3FF4AC0F4FF040EE15C7F
:1070E60002E2E16AE552E16EE552E5CFDAFFE7CF6B
:1070F600D9FF12003EC048F03DC047F03D50420265
:10710600F4CF3CF0F3CF3BF03E504302F4CF3EF0D9
:10711600F3CF3DF04202F3503C26F4503D22E86A9C
:107126003E2247504302F3503C26F4503D22E86A83
:107136003E2243AEA3EF38F047503D5E48503E5ADC
:1071460048AE000C42503D5E43503E5A000C3DC0D6
:1071560047F03D504202F4CF3CF0F3CF3BF03E50B7
:107166004302F4CF3EF0F3CF3DF04202F3503C260B
:10717600F4503D22E86A3E2247504302F3503C2633
:10718600F4503D22E86A3E22000C12010002020081
:107196000040D80492FD8201010200010902430069
:1071A600020100C0320904000001020201000524A8
:1071B6000010010424020205240600010524010032
:1071C600010705820308000209040100020A000003
:1071D6000007050302400000070583024000000483
:1071E60003090418035300630068006D0061006C16
:1071F600007A0048006100750073001603450069B7
:107206000042006F00740042006F0061007200646B
:0972160000A271E571E971017239
:10722000D9CFE6FFDACFE6FFE1CFD9FFE2CFDAFF31
:10723000FB0EDBCF49F0FC0EDBCF4AF00001800EE5
:107240004A141AE1FB0EDBCFE9FFFC0EDBCFEAFFAD
:10725000EECFF3FFEDCFF4FFEE2A000EEF22F3CFD7
:10726000E9FFF4CFEAFFFD0EDBCFEFFFEF504A6AF4
:10727000F36E4AC0F4FF10D0FB0EDB50FE0806E1AF
:10728000FD0EDBCFE6FF08EC3AF005D0FD0EDBCFBC
:10729000E6FFFAEC0EF0E552E552E5CFDAFFE7CF74
:1072A000D9FF12003B504002F3CF37F0F4CF38F053
:1072B0004102F3503826000EF420396E3B50420252
:1072C000F3503926000EF4203A6E3B504302F3503F
:1072D0003A263C504002F3503826F4503922000E32
:1072E0003A223C504102F3503926F4503A223C50A5
:1072F0004202F3503A263D504002F3503926F450F2
:107300003A223D504102F3503A263E504002F3509B
:107310003A261200FF0EE124E96EFF0EE220EA6E2B
:10732000EDCFF4FFEFCFF3FFF46607D0600EF36408
:1073300004D07B0EF36001D0F39A1200F36AF46A72
:10734000FF0EE124E96EFF0EE220EA6EED6607D043
:107350002F0EEF6404D03A0EEF6001D0F32A120032
:107360003A6A396A386A376A200EE76ED8903B3637
:107370003C363D363E363736383639363A3640506A
:10738000375C415038584250395843503A5809E315
:107390004050375E4150385A4250395A43503A5A59
:1073A0003B2AE72EE4D712004F4B0D0A000D0A00CE
:1073B000454242763131204542204669726D7761FF
:1073C00072652056657273696F6E20312E392E36C4
:0373D0000D0A00A3
:1073D400C00EF36E00EE00F00E0E01D81200EA604B
:1073E40002D0EE6AFCD7F350E9601200EE6AFCD7D3
:1073F4001DEE00F02DEE00F0F86A369C95EC37F0A7
:107404001FEC3AF003EC37F0FBD71200FF0EE35009
:10741400ADBA04D0B06AAC8EAD8A949CADA2FED74E
:10742400AE6EF36EF46A12003031323334353637CF
:0974340038396162636465660089
:10743E001200FEFF0000000000000000000000002F
:10744E00000000000000000000000000000000002E
:10745E00000000000000000000000000000000001E
:10746E00000000000000000000000000000000000E
:10747E0000000000000000000000000000000000FE
:10748E0000000000000000000000000000000000EE
:08749E000000000000000000E6
:087FF800ACF70AFF63F801F089
:00000001FF
